:020000040000FA
:100000000004040000000000041A0000081A0000A8
:100010000C1A0000101A0000141A00000C1B00003B
:100020000C1B00000C1B0000181A00001C1A00001A
:10003000201A0000241A00000C1B0000281A0000DF
:100040002C1A0000301A0000341A0000381A000080
:100050003C1A0000401A0000441A0000481A000030
:100060000C1B00000C1B00004C1A0000501A000072
:10007000541A0000581A00005C1A00000C1B000003
:10008000601A0000641A00000C1B0000681A0000CF
:100090006C1A0000701A0000741A0000781A000030
:1000A0007C1A0000801A0000841A0000881A0000E0
:1000B0000C1B00000C1B00000C1B00008C1A000025
:1000C000901A0000941A0000981A00009C1A000070
:1000D000A01A0000A41A0000A81A0000AC1A000020
:1000E0000C1B00000C1B00000C1B0000B01A0000D1
:1000F000B41A00000C1B00000C1B0000B81A000012
:10010000BC1A00000C1B00000C1B00000C1B0000A4
:100110000C1B00000C1B00000C1B00000C1B000043
:10012000C01A00000C1B00000C1B0000C41A0000C9
:10013000C81A0000CC1A00000C1B00000C1B0000A9
:100140000C1B00000C1B0000D01A00000C1B000050
:100150000C1B00000C1B00000C1B0000D41A00003C
:100160000C1B00000C1B00000C1B0000D81A000028
:10017000DC1A0000E01A0000E41A0000E81A00008F
:10018000EC1A0000F01A0000F41A0000F81A00003F
:10019000FC1A0000001B0000041B0000081B0000EC
:1001A0000C1B00000C1B00000C1B00000C1B0000B3
:1001B0000C1B00000C1B00000C1B00000C1B0000A3
:1001C0000C1B00000C1B00000C1B00000C1B000093
:1001D0000C1B00000C1B00000C1B00000C1B000083
:1001E0000C1B00000C1B00000C1B00000C1B000073
:1001F0000C1B00000C1B00000C1B00000C1B000063
:10020000FFFFFF00FFFFFF00C8040000C80400005C
:10021000C8040000C8040000C8040000C8040000AE
:10022000C8040000C8040000C8040000C80400009E
:10023000C8040000C8040000C8040000C80400008E
:10024000C8040000C8040000C8040000C80400007E
:10025000C8040000C8040000C8040000C80400006E
:10026000C8040000C8040000C8040000C80400005E
:10027000C8040000C8040000C8040000C80400004E
:10028000C8040000C8040000C8040000C80400003E
:10029000C8040000C8040000C8040000C80400002E
:1002A000C8040000C8040000C8040000C80400001E
:1002B000C8040000C8040000C8040000C80400000E
:1002C000C8040000C8040000C8040000C8040000FE
:1002D000C8040000C8040000C8040000C8040000EE
:1002E000C8040000C8040000C8040000C8040000DE
:1002F000C8040000C8040000C8040000C8040000CE
:10030000C8040000C8040000C8040000C8040000BD
:10031000C8040000C8040000C8040000C8040000AD
:10032000C8040000C8040000C8040000C80400009D
:10033000C8040000C8040000C8040000C80400008D
:10034000C8040000C8040000C8040000C80400007D
:10035000C8040000C8040000C8040000C80400006D
:10036000C8040000C8040000C8040000C80400005D
:10037000C8040000C8040000C8040000C80400004D
:10038000C8040000C8040000C8040000C80400003D
:10039000C8040000C8040000C8040000C80400002D
:1003A000C8040000C8040000C8040000C80400001D
:1003B000C8040000C8040000C8040000C80400000D
:1003C000C8040000C8040000C8040000C8040000FD
:1003D000C8040000C8040000C8040000C8040000ED
:1003E000C8040000C8040000C8040000C8040000DD
:1003F000C8040000C8040000C8040000C8040000CD
:100800000FA220000E7F24000E01880000000000CF
:10081000000020000000E000020032000001200083
:1008200020028800140007005B0007000000E000C1
:1008300003003A0080682100010020000200370018
:100840000000200001002000810F70000100320034
:1008500014000700000020000000E0000200320049
:100860000000020000000000DC1402000000000094
:100870000040DA000000FE004440A90040112000C2
:100880000000E0000300320000002000A00188000A
:100890004440A800000006008A1F78008B1F7800E3
:1008A0000000060091018800800478000000EB0041
:1008B0001A003700E284440032A0B4009905BA005F
:1008C000E284440032A0B4009906BA00E2844400F5
:1008D00032A0B4000006EB00476FDE00FD07B20057
:1008E000636CE10003003A00EBFF07000000EB003F
:1008F0000A003700606CE10004003A00005DEB0084
:100900008B05E900FDFF3E00040037006168E1004F
:10091000010032000086EB000B00070019C7BA0087
:100920001905BA000E04E00003003A000A00E000D6
:10093000E0FF3A0000000600FE07B2009E018800BA
:100940008A047800F5FF3700395DBA008B05E900AD
:100950000C003200295DBA008B05E9000800320066
:100960000C00E00003003A00E284440032A0B4002E
:10097000F5FF370019DDBA008B05E900FAFF3A00F0
:100980008904E800E184440032A0B40000000600BD
:100990000040DA000000FE00000005008001780041
:1009A00002003700815978000201E9000200E000EE
:1009B000FCFF3A00000006001201000000020000E7
:1009C0000000000000080000D80400003C00000007
:1009D0000001000001020000000100000902000007
:1009E000290000000101000000C0000032090000E1
:1009F00004000000000200000300000000000000EE
:100A0000092100001101000000010000221D00006A
:100A10000007000005810000034000000001000005
:100A20000705000001030000400000000100000075
:100A30000403000009040000340300004D0000001E
:100A40006900000063000000720000006F000000F9
:100A500063000000680000006900000070000000F2
:100A6000200000005400000065000000630000004A
:100A7000680000006E0000006F0000006C000000C5
:100A80006F000000670000007900000020000000F7
:100A9000490000006E000000630000002E0000000E
:100AA0002603000055000000530000004200000033
:100AB0002000000048000000490000004400000041
:100AC00020000000420000006F0000006F000000E6
:100AD000740000006C0000006F0000006100000066
:100AE00064000000650000007200000006000000C5
:100AF000FF09000001A10000011900000129000008
:100B00004015000000260000FF00000075080000EE
:100B100095400000810000001901000029400000FC
:100B200091000000C0000000EE8400001885000065
:100B30001C850000508500004572000061730000B4
:100B4000696E0000672000004465000076690000BF
:100B5000636500002E2E00002E000000457200008C
:100B60006173000065200000436F00006D7000009D
:100B70006C65000074650000005700007269000099
:100B800074650000204300006F6D0000706C000071
:100B900065740000650A0000507200006573000073
:100BA00073200000526500007365000074000000AF
:100BB000526500007365000074000000754D000070
:100BC0004F470000493200000A4200004F4F00002A
:100BD000544C00004F41000044450000520000000A
:100BE0000080FB008181FB00000140000281410088
:100BF0004311DD0003A020000301410012F0A10019
:100C00000104E00004003A0000004000A180200040
:100C1000823078000300370000004000E1802000AF
:100C20008230780012E0A1006401410012E0A000CF
:100C300000000600214A800080C0B300E78F50000A
:100C40000E003E0001407800818120009140780034
:100C50000104E00004003A0013C0B30082812000C8
:100C60000349780005003700E1CF500003003A0047
:100C700023C0B30082812000034978004194200002
:100C80000081FB00910811007140800080487800CD
:100C9000A1952000D1408800219420009100780087
:100CA000E1806000030032000004E0000C003A0024
:100CB000000006000004E000110032000294200051
:100CC00092017800D140800093587800D14088008C
:100CD0000309E8000040E900F8FF3A0000000600C0
:100CE0000294200092017800D1408000935878004F
:100CF000D14088000309E8000040E900F8FF3A000D
:100D00000000060000C8B30021952000914F10009C
:100D100033003A0001CCB300209420000148780051
:100D20005095200010407800E24F5000090032003A
:100D3000E34F500019003200E14F500026003A0006
:100D4000C04D2800004A880020012000204A880069
:100D500000000600409520001004E0000C003A005E
:100D60001080FB000000400041592800610078001D
:100D7000004A880041942000204190008248780079
:100D80008100E800304090008048780000000600B4
:100D9000209420000048EB00000006004095200051
:100DA00021C0B30090CF100008003E001080FB006F
:100DB000000040006159280061007800004A880066
:100DC0001080FB00204A88000000060020942000CC
:100DD0000048EB0000000600209420000048EB00D3
:100DE000000006000040EB00A1952000804878003C
:100DF0008100E800804878002095200010407800AD
:100E00007F4060000080FB00E10F50000B003200CB
:100E1000E20F50000C0032000000E00028003A0011
:100E2000209420001070A0000348E200240032004B
:100E30000100E9001014A0002100370020942000D8
:100E40001070A0001E003700209420001070A00039
:100E500060952000104078006F406000180032005C
:100E6000609520001004E000070035001040780075
:100E70006F4060000080FB0000004000A180200067
:100E8000E1007800070037006095200010407800EE
:100E90006F4060000080FB0000004000E180200007
:100EA000E10078000040280091006000808F500031
:100EB00003003A0011C0B300A0952000014878005B
:100EC000000820002194200011006000070032007B
:100ED000A0952000004A8800010078001000A000C2
:100EE00021C0B3000080E80001487800000006003F
:100EF000AA24AB0011003200A040800010419000F5
:100F000001C8B300814F51000B003A0071408000CE
:100F10001141900041C8B300814F510006003A00D2
:100F2000C1C0B30011409800A040800090409000E4
:100F30000174A00011409800AA24A9000008200014
:100F40005024880000000600881F78007040800050
:100F5000100478004E44DE00614464000020A200CA
:100F60007040880030408000E80F50000B003A00CD
:100F7000409520001080FB00F007B200B0248800EC
:100F80009604E20003003200000120003040880097
:100F900002003700400020003040880019C8BF0020
:100FA000E14F500021003A00A195200070408000E0
:100FB000110098001FFF070018C8BF00E24F500043
:100FC00008003A0041C0B300704080001140980012
:100FD00070408000904090000174A0001140980083
:100FE000200037000804E00008003A0081C4B30084
:100FF0007040800011409800704080009040900048
:101000000174A000114098001600370081C0B300A1
:101010007040800011409800704080009040900027
:101020000174A000114098000E0037008094200049
:101030001004E0000A003D00514A8000C808DE00AC
:10104000640040001080FB004800DD00008070005C
:101050000100320000000100809420001070A10007
:101060001968EF004F047800000006000468EF00E4
:101070000001EB008200780040072000ED0507002A
:101080008284A90000012000002488000968EF0084
:10109000000006008284A80000012000502488007F
:1010A00010C0B30004E8B7000968EF000001EB00CE
:1010B0008200780050072000DE053700889FBE00C0
:1010C0004095200011C0B30090CF10000E003A00F0
:1010D0000080E900104078007F4060000A003A007C
:1010E000209420001070A0003095200032C0B30082
:1010F000904F110003003A000140780003E8B70068
:10110000010037000368EF00409520001004E00064
:101110009C003A000080E900104078007F406000A9
:10112000E24F500097003A00609520001040780090
:101130006F406000930032006095200010407800FE
:101140006F4060000080FB00E10F50008D003C000C
:10115000000220000608E3008A003A0020942000E4
:101160001070A000609520001004E0000C00350015
:1011700010417800EF4061008180FB0081804000D9
:10118000A280200062847800104078006F406000E8
:101190000080FB0001952000E14478000C0037003E
:1011A0006095200010417800EF4061008180FB00D5
:1011B00081804000E2802000628478001040780046
:1011C0006F4060000080FB00E1942000E144780063
:1011D0000908A30002003A000820A100010037001E
:1011E0000820A000609520001004E00007003500F2
:1011F000104078006F4060000080FB00000040005D
:10120000A18020008830780007003700609520001A
:10121000104078006F4060000080FB00000040003C
:10122000E1802000883078003095200031C0B30084
:1012300090CF10001A003A001800E00013003D00A3
:10124000630040001004E000080035001040780002
:101250006F4060000080FB00019520006141780034
:101260000214A0008270780008003700609520000A
:10127000104078006F4060000080FB00E194200087
:10128000614178000214A0008270780098409000BC
:1012900040C8B30000C07000104498003900370007
:1012A000880078000120A2001100E00008003D0045
:1012B000114090000074A1000064A00090409800CC
:1012C00022002000500020005A05070003003700CC
:1012D000114090000064A000904098000918A300FD
:1012E00002003A001800E0001B003D00609520005D
:1012F0001004E00008003500104078006F406000E6
:101300000080FB0001952000614178000214A100DB
:101310008270780008003700609520001040780047
:101320006F4060000080FB00E19420006141780084
:101330000214A1008270780018409000B043B200FF
:1013400010449800220020008800780050002000FF
:10135000380507000300370018409000B043B20082
:101360001044980060952000104078006F406000A5
:101370000080FB0000004000A14A20000100400066
:101380001014A1004F04BE0000000600881F780062
:10139000209420001070A000AC24EF0008A02000D2
:1013A000020220008000EB00080078007BFD0700AF
:1013B0009424A8000040EB00E194200080487800CD
:1013C0000195200080487800F19420008048780042
:1013D00011952000804878001268EF009424A9003D
:1013E0006800440070408800A8408800B840880029
:1013F000409520001040780008E8B7000004E000A5
:1014000003003A0000012000304088000600370049
:1014100012002000818020000200780005050700EE
:1014200000022000304088004F04780000000600D1
:101430002095200001C6B30010C060003F003A00B4
:10144000309520001080FB008000EB00EB0F500077
:10145000E08F580039003E00006001001C0037009A
:101460001C003700350037001A0037003300370002
:10147000060037000A0037002C0037000A0037004A
:1014800008003700140037002000370020942000A7
:101490001070A0008000200030408800000006008E
:1014A00018FE3700B9FF370080802000004A88000E
:1014B000209420009000780013C0B3000081E80061
:1014C000034978001108B300010878000000060005
:1014D00044FE3700F9FE3700609520001081FB00C4
:1014E0002181200000942000010841000080E800D4
:1014F0009000780013C0B3000081E8000349780031
:101500001108B300010878000000060020942000B4
:101510001070A000609520009080FB0020812000CA
:101520004295200092707800000006000001EB0058
:101530008200780020002000BE04070000000600A2
:101540009EC0A9000080EB00702488005024880011
:10155000AA24EF00AC24EF002000200030258800F2
:10156000A824EF008644A900F00920008024880008
:101570006024880082C4A8008804A80000A020007D
:10158000C800DE00C12488000008EB00301078009D
:101590006000B8002050880031508800405088001A
:1015A0005150880060508800715088008050880039
:1015B00091508800A0508800B1508800C050880029
:1015C000D1508800E0508800F15088009424A80091
:1015D0009624EF0094A4A9009424A9008000200080
:1015E000502488008A64AB00FCFF3A000040EB0006
:1015F0002194200080487800819420000081FB0025
:10160000820878008180E80002F02F0091086100D4
:1016100013C0B30002822000034978001282200028
:10162000034978000268EF000068EF000468EF00EB
:101630000A28EF00E19420008048780001952000FE
:10164000804878001028EF000C28EF00F19420006B
:1016500080487800119520008048780080A0200004
:1016600070408800D0002000502588002095200080
:101670001050880081C0B30000A02000014878000D
:101680000000E80041C0B300014878001074A000D9
:101690000868EF002228EF002428EF000968EF0017
:1016A0000628EF0000000600889FBE008A1F780011
:1016B00000457800814478000984FB000838A300C5
:1016C000030032008040EB000A40780044FD070030
:1016D0000828A3000300320011C0B3000A407800BC
:1016E0003FFD07000A85FB000A054500A04A2000CF
:1016F00009707D004F0578004F04BE000000060011
:101700000104E000050032000082FB0004024200F8
:10171000E580200065027A00040037000082FB00AB
:1017200004024200A580200065027A008002EB00DE
:101730000400E0001A00320012029800034A780008
:10174000144190000244B2001242980014419000EB
:101750000234A00012429800144190000274A000CC
:10176000124298000104E000070032000080FB00F4
:1017700000004000E1802000008040001020A20016
:1017800084027800060037000080FB000000400063
:10179000A1802000008040001020A2008402780078
:1017A00005007800000006000004E00014003A0084
:1017B00081C0B300B040800001487800B040800094
:1017C0002195200011009800C1C0B300114098007D
:1017D000B0408000904090000174A000114098003B
:1017E00041C0B300704080001140980070408000FC
:1017F000904090000174A000114098000000060085
:101800008180FB000080FB00000040000080400061
:101810004300DD0002A0200082014000134290003E
:1018200041C8B30001427200944198006400400036
:10183000020040001041900081407100114098006A
:101840000000060094A4AB00190032000080FB00E9
:1018500000004000E18020000080400090007800FF
:101860001103BE00040420000500200006036200EE
:101870008003EB008688BE00900078001103BE0054
:1018800084186B0085906B00900078000120A20006
:1018900001087800914190000344B2009340980001
:1018A000100078009040900004C168001240980039
:1018B000000006002048E2002A003A0010C0B300F1
:1018C00020E8B7002148E20026003A0021E8B700EE
:1018D00019C8BF00E24F50000A003A007040800073
:1018E0000048EB0081C4B3007040800011409800B4
:1018F00070408000904090000174A000114098005A
:1019000000000600E14F500016003A001E68EF008C
:1019100080C0B300A140800080487800A2408000D1
:10192000219520001101980043C0B3001341980095
:10193000A2408000924190000374A00013419800DF
:1019400014C0B300E381200084497800B2408000D5
:1019500000497800B04080001100980001C8B30031
:101960001140980000000600A0408000104278005E
:10197000414A8000C808DE00A09420001080FB00CF
:101980004800DD00008070008480FB00808F5000E4
:1019900001003600004278008480FB000100500006
:1019A000819420004801DD00F30F20009181610047
:1019B000828871004800DE008180E800804878005D
:1019C0000404E000090032000000EB0061942000F4
:1019D00011017800A3952000634978008208E8008F
:1019E0000000E800804F5200F8FF3E00414A8000AE
:1019F000C808DE00A09420001080FB004800DD0035
:101A0000008070001900320081C0B300B040800037
:101A100001487800A1952000B04080001100980096
:101A2000A040800010E8A30008003A0081C4B30081
:101A3000B040800011409800B0408000904090007D
:101A40000174A000114098000000060081C0B3009E
:101A5000B040800011409800B0408000904090005D
:101A60000174A000114098000000060081C0B3007E
:101A7000B040800001487800B040800021952000EF
:101A80001100980041C0B30011409800B0408000A0
:101A9000904090000174A00011409800514A8000CD
:101AA000C808DE00C09420001080FB004800DD0064
:101AB00000807000010032000000010080942000CE
:101AC0001070A1000148E20001003A0079FF070010
:101AD0000000060019C8BF00E24F500001003A00A4
:101AE000A1FF37001968EF001E48E2000D003A0020
:101AF00081C0B300B040800001487800B040800051
:101B00002195200011009800C1C0B3001140980039
:101B1000B0408000904090000174A00011409800F7
:101B2000000006001E68EF00000006000268EF00DB
:101B30000068EF0019C8BF00E24F50000D003A00E6
:101B400081C0B300B040800001487800B040800000
:101B5000A19520001100980081C4B30011409800A5
:101B6000B0408000904090000174A00011409800A7
:101B700000000600809520001080FB009195200059
:101B80009180FB00C808DD008100700040942000B7
:101B9000908F500007003100809520009080FB005E
:101BA0000000E8001081FB004811DD004094200097
:101BB000010871001FFC0700A19520007040800003
:101BC0001100980081C4B30070408000114098005B
:101BD00070408000904090000174A0001140980077
:101BE0000000060094A4A900000820002194200011
:101BF000110060001F003A00809420001004E000F3
:101C000008003D0020C0B30019E8B7000048E2001A
:101C100001003A00C5FF07002168EF002068EF00CF
:101C20000000060081C0B300B04080000148780089
:101C3000B04080002195200011009800C1C0B30081
:101C400011409800B0408000904090000174A000C6
:101C50001140980041C0B3007040800011409800CE
:101C600070408000904090000174A00011409800E6
:101C700000000600209520001004E0000A003D004E
:101C800010C0B30019E8B7000248E20001003A00B2
:101C9000A6FF07002168EF002068EF000148E2007E
:101CA00014003A0003FF370020C0B30019E8B70062
:101CB00081C0B300B040800001487800B04080008F
:101CC000219520001100980041C0B30011409800F8
:101CD000B0408000904090000174A0001140980036
:101CE0002168EF002068EF000148E20001003A009F
:101CF000F0FE0700000006001868EF000168EF0022
:101D00000268EF000068EF001E68EF001968EF003E
:101D100070408000904090000174A1001140980034
:101D2000704080000020A200704088009040900029
:101D30000174A100114098000E48AA00B040800034
:101D4000904090000174A100114098002094200060
:101D50000048EB008000EB00214A880080942000BE
:101D60008180FB00010878000080E80001F02F006E
:101D700010886000AEFD07000001EB0082007800D3
:101D800030002000AB02070096FF3700D0C2B3003E
:101D90001FE8B700C1812000914078000100780061
:101DA000B00FB20013003A00C10FB20000A0200033
:101DB00080804000A1408800010078000020A2003F
:101DC000B040880002C023001101610000402300E0
:101DD000800F510006003A0011009000219520006C
:101DE00007000900B05878008000B100C2FF37003A
:101DF00038FF3700E80F500001003A0052FC07009E
:101E00000000060010418000214180006100400078
:101E1000E080480010418800214188000448E20029
:101E200004003A000948EC0009E8B70001003A0054
:101E300009E8EF0000000600881F780030408000AD
:101E40000000E00012003A009424EF008C24EF0020
:101E50002000200030258800A824EF008644A90037
:101E6000F0092000802488006024880082C4A80033
:101E70009404AB0003003A009404A8009404AB005F
:101E8000FDFF3200100020003040880002003700C3
:101E9000E10F500008003A0094C4AB0006003A007D
:101EA0008AA4EF008C24EF008C04A8008C84A80086
:101EB00020002000304088008084AB000500320004
:101EC0008284AB000300320000012000002488005F
:101ED00066FC07008824AB00020032008EC0A90017
:101EE000690037008A04AB00070032008C04AB00A5
:101EF0000500320092FD07004000200030408800BD
:101F000010002000502488008A84AB0003003200B7
:101F10008C84AB00010032005EFC070080C4AB0083
:101F2000030032000004200000248800B5FF0700F1
:101F30008A44AB000E0032008C44AB000400320037
:101F4000120020008000EB0030072000390207005B
:101F500040002000502488001FC8BF00030032004A
:101F60000040E9001FE8B70001003A0051FE0700F9
:101F70008AE4AB00030032008CE4AB0001003200C5
:101F8000DBFB07008A24AB00090032008C24AB0085
:101F900007003200120020008000EB00F0FF270055
:101FA000240207008EA4EF002000200050248800A7
:101FB00030408000E30F500002003E008EC0A900B8
:101FC000310037008C64AB002E00320048C0B300F3
:101FD0008A64AB0003003A002A0037008A64AB0031
:101FE0002800320091248000C08120000148780040
:101FF0000181FB004411DE000240780002427800BB
:10200000D381200084497800820020005224880077
:102010000138A30009003A008080FB0002952000EF
:10202000E2C1780061C261000404A2000304A100BF
:1020300084C1710003F17800080037008080FB0044
:10204000E2942000E2C1780061C261000404A200B1
:102050000304A10084C1710003F178000004E000D2
:1020600002003A0049FF0700040037000001EB00BE
:10207000C181200020072000EE0107000844E9008C
:10208000D6FF3A008EC0A9004F0478000000060079
:10209000104180002141800000000600881F780068
:1020A0002628EF002828EF0090CAB3002AE8B700DE
:1020B00000802A00604188002000200070418800D4
:1020C00018C0B30008407800818320008848780059
:1020D0003068EF0034A8EF0036A8EF003268EF0058
:1020E000D1C1B30070FD070003C4B300028C20000F
:1020F0008040EB000840780081FD070030418800F7
:102100004F0478000000060012832000124178007E
:102110000281FB008001EB004A18DD00C610DE00E2
:10212000810070004A10DD0022042400023B880078
:102130008141780022032000034978000081EB00F0
:102140000208BB001000FC0050052000303B880056
:10215000A00A2000303B880061E7A80000000000D2
:10216000000000006007E200FEFF350000000600EE
:1021700030002400003B880032C8BF001D00320040
:10218000019020000081FB008001EB00A441800051
:10219000B54180000201520083815A000342780059
:1021A0002003200004487800020078001108BB00DA
:1021B000110190000288BB001000FC0050052000B7
:1021C000303B8800A00A2000303B880061E7A8006F
:1021D00000000000000000006007E200FEFF350084
:1021E00032C8ED0032E8B700E48040000004E000AF
:1021F000E4FF3A0061C7A9000000060023032000A5
:1022000093417800400ADE00050020000443780076
:102210002203200006497800000178001282BA00EB
:10222000840078001200BA000342780022032000E4
:102230000449780000000600889FBE008A9FBE0007
:102240003048E20022003A00404180000000E000F7
:10225000020032001000E0007301350030418000C0
:102260000000E00005003A00F08B2000F183200020
:102270000204200000014100030037001000E000CC
:10228000F9FF3D0068013700D0687800820F5000E8
:10229000FDFF3A0003C4B300028C20008040EB0035
:1022A00010C0B30016FD07003041880010C0B30015
:1022B00030E8B700F0872000010420008080400053
:1022C0000068EB00810F5000FDFF3A005601370017
:1022D0000084200010407800E54F5000910032004B
:1022E00006003E00E34F50005A0032006E003E00F0
:1022F000E24F50004C013A0006003700E74F500013
:10230000E6003200DB003900E84F500046013A0099
:102310003A01370020C0B3000188200080487800CF
:1023200082C3B3008100E800824878008100E800A1
:102330008048780011C0B300308820000148780040
:102340000040EB00418820008048780082C1B30043
:102350008100E800824878008100E8008048780029
:102360008100E8008048780000802E00F1FF2F00F7
:102370006241800073418000020040008380480079
:10238000F20F200083882000824960004802DE00AE
:102390008301E800844978008301E80082C9600075
:1023A000C808DE000300E800014878000000E800EB
:1023B00000C8EB003848E20019003A0031C0B30011
:1023C000014878000040EB0082CFB300E380410079
:1023D00082487800B2CAB3008100E80082487800E1
:1023E00022C0B3008100E800824878008100E80044
:1023F0008048780082C0B3008100E80082487800FD
:102400008100E800804878008100E800804878007A
:102410008100E800804878000100E80000C8EB0077
:10242000404180000000E000020032001000E000A7
:10243000FD00350003C4B3000288200011C0B300C2
:1024400001407800AEFC0700404188003068EF0092
:10245000F5003700108420001004E00008003A0066
:10246000A0CAB3002AE8B70083BF2A0063418800EE
:1024700023002000734188003868EF00080037000F
:1024800090CAB3002AE8B70000802A0060418800A3
:10249000200020007041880010C0B30038E8B70069
:1024A0003068EF00E00037008000EB0010002000F3
:1024B00010010700C05928005601070060C0B30092
:1024C00031E8B7002AC8BF000080FB000000E80028
:1024D000E60F50000B0034000BFF070056FE07000C
:1024E0003148EC0031E8B7000080FB00A1822000F9
:1024F000914078008180FB008100E800810F50004E
:10250000F5FF350061C7A9003068EF008000EB00DF
:1025100010002000F7000700E05A28003D010700E6
:10252000C1003700A0418000B1418000E10F4000B0
:10253000E08F48000E003A00128420001281FB0058
:10254000238420009381FB00C819DD000300710083
:10255000328420001281FB00438420009381FB0021
:10256000C819DD0083007100A0418800B1418800D6
:10257000128420001281FB00238420009381FB0041
:10258000C819DD0003007100328420001281FB00B5
:10259000438420009381FB00C819DD008300710093
:1025A000A2418000B3418000820F5000838F580009
:1025B0002E003A005084200010407800E14F500077
:1025C0002A0036000044EB0021832000914078006F
:1025D0000181FB00820141000080FB00820320009A
:1025E000000051004F01DE00000041000081D100D9
:1025F0000880FB0000004100640040000000400033
:1026000002842000624278000482FB000000410046
:10261000104190004811DD0002017200009020007E
:1026200002B079000140E80032E8B700A241800022
:10263000B341800061014100E0814900A24188006E
:10264000B3418800FC4F500001003A00C8FE07006B
:102650000844E80050842000104078008080FB008F
:102660008100D100814F5400D7FF39003068EF005E
:102670006D003700BEFE070034A8EF0036A8EF005B
:102680003068EF008000EB00100020009900070088
:10269000D05B2800DF000700630037004041800066
:1026A0000000E000020032001000E0005E00350093
:1026B00071C0B30000882000014878001284200017
:1026C0001281FB00238420009381FB00C819DD00E8
:1026D00003007100328420001281FB00438420003B
:1026E0009381FB00C819DD0083007100F20F200008
:1026F00013882000824960004802DE008301E80060
:10270000844978008301E80082C96000C808DE00BF
:102710000300E80001487800508420001040780051
:102720008380E80080487800E14F50002B0036009D
:102730000044EB000881FB008001EB0014842000C2
:102740001482FB00258420009582FB00C82ADD004E
:1027500005007200348420001482FB0045842000B0
:102760009582FB00C82ADD0085007200020040004F
:1027700083804800A1FE07008884FB005484200069
:102780009482FB008502D1008583FB0007855400FD
:102790000A02B000068820000A0545000A05430029
:1027A000F40F2000044D6000C805DE001B459800B2
:1027B00081016200078054001002B0000000400058
:1027C0000000430004C86100C818DE0011409800F2
:1027D00008C4E80088CF5200D6FF3E0003C4B3000F
:1027E0000288200011C0B30001407800C4FB07003C
:1027F000404188003068EF000B0037008000EB009C
:10280000100020003B000700805D280081000700C9
:102810009424EF000080EB00000000000000E900BD
:10282000FDFF3A000000FE004F05BE004F04BE0051
:102830000000060031072000810F50000D0032001B
:1028400005003C00E10F500010003200E30F500083
:1028500011003A000F00370041072000810F50009F
:10286000080032008100E800810F50000A003A00A1
:1028700002003700FE00070007003700FC000700D9
:1028800005003700FA0007000300370003FE0700C9
:10289000010037007100070010000500EC22A800BD
:1028A000000000000000000000000000EC22A90071
:1028B0000000060000F02F00E022B600F002A900A0
:1028C000F022A900E822A900F402A900F422A9003C
:1028D000EC22A900000006000000FB0001F02F0020
:1028E000221780008280600080807000211788009D
:1028F0000000060080417800F00F2000E022B700C1
:10290000F422A800F402A900EC22A80000000000B4
:10291000000000000000000012178000EC22A90057
:102920000278A300F8FF3A0002F02F00002E2000EA
:1029300010086100F422A9008180FB008100EA00F8
:10294000CF08DE00A21780000200A1000281700003
:10295000A217880003407800DFFF0700CFFF370091
:10296000D4FF070000202100A10720001801070064
:102970008040EB0080C3B300DEFF07008040EB0027
:1029800080C0B300DBFF07008040EB0010C0B30045
:10299000D8FF07008040EB0060C0B300D5FF070000
:1029A0008040EB00C0C0B300D2FF070000B82B008E
:1029B0000100200006013700F0F32F004427B60085
:1029C00042A7AB0003003A000000000042A7AB00A2
:1029D000FDFF320040A7A900F0C2A900D022A80044
:1029E000DFFF07000000EB00E3000700D4FA070058
:1029F0000060FE0010FD070030408000FF0F500017
:102A0000FBFF36008824AB00F9FF3A000AFE0700FE
:102A1000F7FF3700881F780000047800184078001E
:102A20000004E0000B003200EA4F500004003A00BE
:102A30008040EB0000CCB300AEFF0700020037007F
:102A400011C0B300ABFF0700584078000004E0005D
:102A5000F5FF3A004F0478000000060020952000A2
:102A6000104078007F406000E14F500054003A0071
:102A7000609520001004E00051003A00630050000F
:102A800061C0B30090CF10001B003A000080E80046
:102A900010407800FBC04000814F5000040032001D
:102AA0008140E800814F500013003A000B003700CE
:102AB00008C8BF00E14F50000F003A000050280046
:102AC000004A880090002000204A880001CCB30012
:102AD0002094200001487800070037006057280044
:102AE000004A8800D0012000204A880001CCB300B1
:102AF00020942000014878002095200002C6B300F1
:102B00009040610000C2B30080CF50002C003A001A
:102B10003095200010407800E34F5000190032003B
:102B200003003E00E24F500025003A000500370048
:102B3000EA4F50000B003200EB4F500020003A00EB
:102B400018003700A0832000004A880010002000F1
:102B5000204A880011CCB30020942000014878005E
:102B60000000060001C8B30020942000014878004E
:102B70005095200010417800A18320008248780001
:102B800000000600B0832000004A880010002000EA
:102B9000204A880011C8B300209420000148780022
:102BA0000000060001C8B30020942000014878000E
:102BB0004095200010417800B183200082487800C1
:102BC00000000600E10F500003003200E20F500049
:102BD00004003A0002003700F4C2A800000006001A
:102BE000F4E2A80000000600E10F500003003200EC
:102BF000E20F500004003A0002003700F4C2A900BE
:102C000000000600F4E2A90000000600E10F5000F9
:102C100003003200E20F50000B003A0005003700BD
:102C200000042000F402B6000000EA004F00DE00BD
:102C30000000060000082000F402B6000000EA00D0
:102C40004F00DE000000060000000500E10F50000C
:102C500003003200E20F500004003A000200370087
:102C6000F0C2A90000000600F0E2A9000000060082
:102C70008824AB000200320010002000DAFF370089
:102C8000000220000608E30010003A00F041800036
:102C9000E10F500002003A00CAFF07001A00370097
:102CA000B1042000810F500003003A001000200002
:102CB000CDFF07001400370061092000810F50008C
:102CC000110036003E28EF000F003700F041800071
:102CD000E10F500002003A00BAFF07000A00370077
:102CE00021032000810F500003003A001000200053
:102CF000BDFF070004003700613B2000810F50003A
:102D0000010036003E28EF003E28EC0000000600DF
:102D10004009000022000000000000000008000040
:102D20002600000000000000000A00002000000053
:102D3000000000003A08000002000000000000004F
:102D4000400800000001000000000000260800000C
:102D500014000000000000003C0800000200000019
:102D600002000000010000003E0800000200000018
:102D700000000000000000000000E00013003A0026
:102D800083E0A800100020002700070010002000AA
:102D90001D0007000004E00006003A003008200093
:102DA0004007B6000300320083E0A900001A0400C7
:102DB00000000000E05D280016FF07001000200062
:102DC000A2FF070020002000A0FF0700000006006F
:102DD000F03FB1000180B10006003500EE030900AC
:102DE00000000000403FB1000180B100FBFF3D004A
:102DF0001000B000203FB000020035000080090044
:102E00000000000000000600E10F500005003A003D
:102E100090168000620060000000E9004F00DE00B4
:102E20000000060000000500E10F500001003A001C
:102E3000D022A80000000600FFFFFF00FFFFFF00F8
:10340000101B040000000000F41B0400000000007A
:10341000F41B040000000000F41B04000000000086
:10342000F41B040000000000F41B04000000000076
:10343000F41B040000000000F41B04000000000066
:10344000F41B040000000000F41B04000000000056
:10345000F41B040000000000F41B04000000000046
:10346000F41B040000000000F41B04000000000036
:10347000F41B040000000000F41B04000000000026
:10348000F41B040000000000F41B04000000000016
:10349000F41B040000000000F41B04000000000006
:1034A000F41B040000000000F41B040000000000F6
:1034B000F41B040000000000F41B040000000000E6
:1034C000F41B040000000000F41B040000000000D6
:1034D000F41B040000000000F41B040000000000C6
:1034E000F41B040000000000F41B040000000000B6
:1034F000F41B040000000000F41B040000000000A6
:10350000F41B040000000000F41B04000000000095
:10351000F41B040000000000F41B04000000000085
:10352000F41B040000000000F41B04000000000075
:10353000F41B040000000000F41B04000000000065
:10354000F41B040000000000F41B04000000000055
:10355000F41B040000000000F41B04000000000045
:10356000F41B040000000000F41B04000000000035
:10357000F41B040000000000F41B04000000000025
:10358000F41B040000000000F41B04000000000015
:10359000F41B040000000000F41B04000000000005
:1035A000F41B040000000000F41B040000000000F5
:1035B000F41B040000000000F41B040000000000E5
:1035C000F41B040000000000F41B040000000000D5
:1035D000F41B040000000000F41B040000000000C5
:1035E000F41B040000000000F41B040000000000B5
:1035F000F41B040000000000F41B040000000000A5
:10360000F41B040000000000F41B04000000000094
:10361000F41B040000000000F41B04000000000084
:103620000F0221000E7F24000E0188000000000020
:10363000000020000000E000020032000001200035
:103640002002880014000700690007000000E00065
:1036500003003A00000828000100200002003700A3
:103660000000200001002000810F700001003200E6
:1036700014000700000020000000E00002003200FB
:103680000000020000000000CC80020000000000EA
:103690000040DA000000FE004440A9004012200073
:1036A0000000E0000300320000002000A0018800BC
:1036B0004440A800000006008A1F78008B1F780095
:1036C0000000060091018800800478000000EB00F3
:1036D0001A003700E284440032A0B4009905BA0011
:1036E000E284440032A0B4009906BA00E2844400A7
:1036F00032A0B4000006EB00476FDE00FD07B20009
:10370000636CE10003003A00EBFF07000000EB00F0
:103710000A003700606CE10004003A00005DEB0035
:103720008B05E900FDFF3E00040037006168E10001
:10373000010032000086EB000B00070019C7BA0039
:103740001905BA000E04E00003003A000A00E00088
:10375000E0FF3A0000000600FE07B2009E0188006C
:103760008A047800F5FF3700395DBA008B05E9005F
:103770000C003200295DBA008B05E9000800320018
:103780000C00E00003003A00E284440032A0B400E0
:10379000F5FF370019DDBA008B05E900FAFF3A00A2
:1037A0008904E800E184440032A0B400000006006F
:1037B000641D0400000000004E1D04000000000015
:1037C000441D0400000000003A1D04000000000039
:1037D000821D040000000000B01F04000000000073
:1037E000001E0400000000000040DA000000FE009F
:1037F000000005008001780002003700B159780010
:103800000201E9000200E000FCFF3A0000000600AF
:103810008001780002003700815978000201E90038
:103820000200E000FCFF3A00000006001201000068
:10383000000200000000000000080000D8040000A2
:103840000900000001000000010200000301000067
:1038500009020000200000000101000000C000007B
:103860003209000004000000000200000806000009
:103870005000000007050000810200004000000029
:1038800001070000050100000240000000010000E7
:1038900004030000090400000A0300004D000000BA
:1038A0006F000000670000006900000034030000A2
:1038B000750000004D0000006F0000006700000070
:1038C0006900000032000000200000004D000000F0
:1038D0006100000073000000730000002000000081
:1038E00053000000740000006F0000007200000030
:1038F000610000006700000065000000200000007B
:103900004400000072000000690000007600000022
:10391000650000001A0300003100000032000000C2
:1039200033000000340000003500000036000000C5
:1039300037000000380000003900000030000000AF
:103940003900000039000000289C0000489C00005D
:103950004C9C0000569C00008A9C00000204000061
:103960000E0100000F1100000F0000000204000013
:103970000E1100001F1000000E00000002040000E5
:103980000C040000040400000E000000020400000B
:103990000E110000111100000E00000002040000D2
:1039A00011110000111300000D0000000A000000BA
:1039B00011110000111300000D000000050A0000A5
:1039C00011110000111300000D000000050A000095
:1039D0000E110000111100000E000000040A00008A
:1039E0000A0A0000111F00000E000000000E000077
:1039F00015170000110E0000000000001C0200005E
:103A000001050000091E00000804000000800000FD
:103A10000402000020000000000000004D690000CA
:103A2000637200006F630000687000004D61000069
:103A30007373000020530000746F00007261000077
:103A400067650000202000002020000030300000CA
:103A500030310000754D00004F4700004932000032
:103A600020500000656E000044720000697600007E
:103A7000650000000200FA00000F780010C0B300DB
:103A80000080FA00000006000200FA00000F780033
:103A9000002020000080FA00000006000200FA006A
:103AA000000F7800F0012000010020000080FA00E3
:103AB000000006000200FA00000F780010C0B300FA
:103AC0000080FA00000006000200FA00000F7800F3
:103AD00020852000900090000100A00011009800B7
:103AE0002085200001202000210098002085200052
:103AF0008000EB0001087800208520000080FA009B
:103B0000000006001200FA005007980062079800B3
:103B100073079800010F98006E019000FE0190005D
:103B2000F001200001002000800F5100818F59001A
:103B3000020036000040EB002F0037002103200078
:103B400091407800614798006E009000FE00900060
:103B500070014000E08148004918DD00C710DE0018
:103B6000810070004910DD001007980021079800BF
:103B70000000EB00000F7800170037001E009000D7
:103B8000AE0090004008DE000040780032E0B70050
:103B90001E0090001000BA0040079800680047001F
:103BA00022002000800078000E08900011FF07001E
:103BB0000E0890000080E800000F98001E009000A2
:103BC000AE00900062004000E080480010079800BE
:103BD000210798001E0FE800F00F20009E007800DB
:103BE000808F5000E5FF3600EE4090002203200059
:103BF0000149780010C0B3000080FA000000060000
:103C00001600FA006007980072079800030F9800EA
:103C1000110F9800445798007E0190008E09900083
:103C2000F001200001002000800F5100818F590019
:103C3000020036000040EB00AB00370032C0BF008E
:103C40000080FB00500798007E0090008E089000D6
:103C500070004000E08048004909DD00C701DE0037
:103C6000830171004901DD0000C02F00F1FF2F002A
:103C700002027800030178008001780001007800DA
:103C800003026200000061008000EB00C000DD0064
:103C9000000020000001BE006120B800000171009A
:103CA0008181710032079800430798000000EB0003
:103CB000000F7800110037003E009000CE00900009
:103CC0004008DE000040780032E0B700C0852000E8
:103CD0001E004000BE0090009100BA00010878006C
:103CE0003E009000CE00900062004000E08048005E
:103CF00030079800410798001E8FE800F03F200031
:103D00009E007800808F5000EBFF36007E00900010
:103D100061006000004078000004E0000300320011
:103D20000020200020079800020037000000EB0070
:103D3000200798000000EB00000F78000B00370010
:103D40002E0090001E0140001E0890009040780058
:103D5000C085200000004100014878001E08900046
:103D60000000E800100F98001E0FE800F01F200070
:103D70009E007800808F5000F1FF36007E0090009A
:103D80008E08900070004000E08048004909DD0086
:103D9000C701DE00830171004901DD0000C02F0072
:103DA000F1FF2F0002027800030178008001780003
:103DB0000100780003026200000061008000EB0057
:103DC000C000DD00000020000001BE006120B8003E
:103DD000000171008181710032079800430798004B
:103DE00020042400003B88003E0090008080EB000F
:103DF0000108BB0050CBB3004100070010002400B5
:103E0000003B88000040EB00204798000000EB00DA
:103E1000000F78002C0037003E009000CE0090008C
:103E20004008DE000040780032E0B700C085200086
:103E30001E004000900078003E0090000108BB008A
:103E40003E009000CE00900061004000E0804800FD
:103E500030079800410798003E0090008000EB007A
:103E60000188BB003E009000CE0090006100400041
:103E7000E080480030079800410798001E8FE80056
:103E80002E40900000C0E800204798002E4090008F
:103E90000004E0000C003D00AE40900000C8B300FC
:103EA00000C04000204798001000FC005005200092
:103EB000303B8800A00A2000303B880061E7A80062
:103EC0000000000000000000F03F20009E0078008D
:103ED000808F5000D0FF36005E00900000407800D8
:103EE00032E0B70010C0B3000080FA000000060006
:103EF0000200FA00000F78000080FA0000000600BF
:103F00000200FA00004F7800360007000004A2000B
:103F10000004E0000D003A0050CBB3009E40780052
:103F200080CF50000B003A001000FC00500520002C
:103F3000303B8800A00A2000303B880061E7A800E1
:103F40000000000000000000030037000000000037
:103F500001003700000000000080FA0000000600A9
:103F60000200FA00000F78000040EB000080FA0029
:103F7000000006000000FA00D1C1B30010C0B30079
:103F800074210700DC2707000080FA00000006000B
:103F90000000FA0010418000FF0F500006003600BC
:103FA00040248000620060000000E00004003A004D
:103FB00074280700030037000000000001003700EC
:103FC000000000000080FA00000006000000FA0077
:103FD0000080EB0060198800092007000080FA00CB
:103FE000000006000000FA0010C0B3000080FA00D4
:103FF00000000600FFFFFF00FFFFFF00FFFFFF00C4
:1040000000000000000000000000000000000000B0
:1040100000000000000000000000000000000000A0
:104020000000000000000000000000000000000090
:104030000000000000000000000000000000000080
:10437000F58B000016EA000000000000800100003C
:104380000100000001070000FFE60000010000003E
:10439000000000001F0000000000000000000000FE
:1043A000000000000000000000000000000000000D
:1043B00000000000000000000000000000000000FD
:1043C00000000000000000000000000000000000ED
:1043D00000000000000000000000000000000000DD
:1043E00000000000000000000000000000000000CD
:1043F00000000000000000000000000055AA0000BE
:10440000EB3C0000904D0000534400004F5300006F
:10441000352E000030000000020100000100000005
:10442000011000000000000000F800000100000082
:104430003F000000FF00000001000000000000003D
:104440001F000000000000000000000029320000F2
:1044500067940000C44E00004F2000004E41000051
:104460004D450000202000002020000046410000B3
:104470005431000032200000202000000000000025
:10448000000000000000000000000000000000002C
:10449000000000000000000000000000000000001C
:1044A000000000000000000000000000000000000C
:1044B00000000000000000000000000000000000FC
:1047F00000000000000000000000000055AA0000BA
:10480000F8FF0000FFFF0000FFFF0000FFFF0000B7
:10481000FF0700008000000009A00000000B00005E
:10482000C00000000DE00000000F000000010000CB
:10483000112000000113000040010000156000007D
:10484000011700008001000019A00000011B0000FA
:10485000C00100001DF00000FF000000000000008B
:104860000000000000000000000000000000000048
:104870000000000000000000000000000000000038
:104880000000000000000000000000000000000028
:104890000000000000000000000000000000000018
:104C0000754D00006F670000693200002020000031
:104C1000202000002008000000000000000000002C
:104C20000011000000110000000000000000000062
:104C30000011000000000000000000000000000063
:104C4000E5450000414400004D45000020200000E3
:104C5000485400004D20000000060000E0710000F4
:104C60004E4F00006253000000000000E079000099
:104C700061530000020000001A0100000000000063
:104C80004220000000490000006E000000660000A5
:104C9000006F0000000F00000072000072000000B2
:104CA0006D00000061000000740000006900000059
:104CB0006F000000000000006E0000000000000017
:104CC0000153000000790000007300000074000030
:104CD00000650000000F0000007200006D00000081
:104CE00020000000560000006F0000006C00000073
:104CF00075000000000000006D000000650000006D
:104D00005359000053540000454D00007E3100000F
:104D1000202000002016000000BF0000B158000055
:104D2000625300006253000000000000B25800000F
:104D300062530000030000000000000000000000BB
:104D400055560000455A0000202000002020000099
:104D50004A5000004720000018460000EE580000AE
:104D6000625300006253000000000000EC58000095
:104D70006253000006000000B32E00000000000097
:104D8000E52E00000048000000540000004D000027
:104D900000000000000F000000880000FFFF00007E
:104DA000FFFF0000FFFF0000FFFF0000FFFF00000B
:104DB000FFFF000000000000FFFF0000FFFF0000F9
:104DC000E55400004D7E000031200000202000004E
:104DD000202000002020000000060000E0710000FC
:104DE0004E4F00006253000000000000E079000018
:104DF00061530000020000001A01000000000000E2
:104E000041520000006500000061000000640000E5
:104E1000006D0000000F0000005F00006500000052
:104E20002E00000068000000740000006D0000000B
:104E30006C0000000000000000000000FFFF000008
:104E400052450000414400004D4500007E31000005
:104E5000485400004D2000000030000000590000C0
:104E60006253000062530000000000002A59000055
:104E70006253000002000000730100000000000007
:104E80000000000000000000000000000000000022
:104E90000000000000000000000000000000000012
:104EA0000000000000000000000000000000000002
:104EB00000000000000000000000000000000000F2
:104EC00000000000000000000000000000000000E2
:104ED00000000000000000000000000000000000D2
:104EE00000000000000000000000000000000000C2
:104EF00000000000000000000000000000000000B2
:104F000000000000000000000000000000000000A1
:104F10000000000000000000000000000000000091
:104F20000000000000000000000000000000000081
:104F30000000000000000000000000000000000071
:104F40000000000000000000000000000000000061
:104F50000000000000000000000000000000000051
:104F60000000000000000000000000000000000041
:104F70000000000000000000000000000000000031
:104F80000000000000000000000000000000000021
:104F90000000000000000000000000000000000011
:104FA0000000000000000000000000000000000001
:104FB00000000000000000000000000000000000F1
:104FC00000000000000000000000000000000000E1
:104FD00000000000000000000000000000000000D1
:104FE00000000000000000000000000000000000C1
:104FF00000000000000000000000000000000000B1
:105000003C680000746D00006C2000006C610000C2
:105010006E6700003D22000068750000223E00001F
:105020000D0A0000093C0000686500006164000092
:105030003E0D00000A090000093C00006D650000FB
:10504000746100002063000068610000727300005A
:10505000657400003D22000075740000662D00009C
:10506000382200003E0D00000A0900000909000076
:105070003C740000697400006C6500003E4500004F
:105080006C6D0000C3A900006C650000746900002D
:1050900020C30000965400003C2F000074690000FB
:1050A000746C0000653E00000D0A00000909000054
:1050B0003C2F000068650000616400003E0D0000A8
:1050C0000A090000093C0000626F000064790000DA
:1050D0003E0D00000A090000090900003C680000BC
:1050E000323E00004D6900006B7200006F760000D8
:1050F000657A0000C3A90000726C0000C591000031
:105100006B200000616C00006B6100006C6D0000A2
:10511000617A0000C3A10000736100003C2F000011
:10512000683200003E0D00000A0900000909000075
:105130003C7000003E4500006C6D0000C3A90000FB
:105140006C6500007469000020C3000096540000E4
:105150003A20000032300000323100002E310000D1
:10516000312E0000303800002E20000028520000B0
:1051700031300000382900003C2F0000703E000054
:105180000D0A000009090000093C0000703E000003
:10519000566500007A65000074C30000A96B00002A
:1051A0006EC30000A9760000207300007A6500003D
:1051B000726900006E7400003A3C00002F7000001D
:1051C0003E0D00000A090000090900003C750000BE
:1051D0006C3E00000D0A00000909000009090000EA
:1051E0003C6C0000693E0000412D00004B3A00007D
:1051F00020310000343A0000313500002D3100002C
:10520000353A000030300000206B0000C3B60000CB
:105210007AC30000B6740000743C00002F6C0000DC
:10522000693E00000D0A000009090000090900009C
:105230003C6C0000693E00004C2D00005A530000F9
:105240003A200000313500003A310000352D0000D1
:10525000313600003A300000302000006BC30000FF
:10526000B67A0000C3B60000747400003C2F000042
:105270006C6900003E0D00000A09000009090000E9
:105280003C2F0000756C00003E0D00000A09000074
:10529000090900003C6900006D67000020730000F0
:1052A000726300003D22000075760000657A000000
:1052B0002E6A000070670000223E00000D0A000008
:1052C000090900003C2F0000626F000064790000B3
:1052D0003E0D00000A0900003C2F00006874000029
:1052E0006D6C00003E0000000000000000000000A7
:1052F00000000000000000000000000000000000AE
:10530000000000000000000000000000000000009D
:10531000000000000000000000000000000000008D
:10532000000000000000000000000000000000007D
:10533000000000000000000000000000000000006D
:10534000000000000000000000000000000000005D
:10535000000000000000000000000000000000004D
:10536000000000000000000000000000000000003D
:10537000000000000000000000000000000000002D
:10538000000000000000000000000000000000001D
:10539000000000000000000000000000000000000D
:1053A00000000000000000000000000000000000FD
:1053B00000000000000000000000000000000000ED
:1053C00000000000000000000000000000000000DD
:1053D00000000000000000000000000000000000CD
:1053E00000000000000000000000000000000000BD
:1053F00000000000000000000000000000000000AD
:105400002E2000002020000020200000202000008E
:10541000202000002010000000BF0000B158000054
:10542000625300006253000000000000B258000008
:1054300062530000030000000000000000000000B4
:105440002E2E000020200000202000002020000040
:10545000202000002010000000BF0000B158000014
:10546000625300006253000000000000B2580000C8
:105470006253000000000000000000000000000077
:10548000427400000000000000FF0000FFFF000069
:10549000FFFF0000FF0F000000CE0000FFFF000034
:1054A000FFFF0000FFFF0000FFFF0000FFFF000004
:1054B000FFFF000000000000FFFF0000FFFF0000F2
:1054C000015700000050000000530000006500007C
:1054D00000740000000F000000CE00007400000007
:1054E000690000006E00000067000000730000000B
:1054F0002E000000000000006400000061000000B9
:105500005750000053450000545400007E31000005
:10551000444100005420000000020000B258000086
:10552000625300006253000000000000B358000006
:1055300062530000040000000C00000000000000A6
:105540004247000000750000006900000064000090
:1055500000000000000F000000FF0000FFFF00003F
:10556000FFFF0000FFFF0000FFFF0000FFFF000043
:10557000FFFF000000000000FFFF0000FFFF000031
:1055800001490000006E000000640000006500009A
:1055900000780000000F000000FF00006500000020
:1055A00072000000560000006F0000006C00000058
:1055B00075000000000000006D00000065000000A4
:1055C000494E000044450000584500007E3100006F
:1055D000202000002020000000C20000B25800007F
:1055E000625300006253000000000000B358000046
:1055F00062530000050000004C00000000000000A5
:10560000000000000000000000000000000000009A
:10561000000000000000000000000000000000008A
:10562000000000000000000000000000000000007A
:10563000000000000000000000000000000000006A
:10564000000000000000000000000000000000005A
:10565000000000000000000000000000000000004A
:10566000000000000000000000000000000000003A
:10567000000000000000000000000000000000002A
:10568000000000000000000000000000000000001A
:10569000000000000000000000000000000000000A
:1056A00000000000000000000000000000000000FA
:1056B00000000000000000000000000000000000EA
:1056C00000000000000000000000000000000000DA
:1056D00000000000000000000000000000000000CA
:1056E00000000000000000000000000000000000BA
:1056F00000000000000000000000000000000000AA
:105700000000000000000000000000000000000099
:105710000000000000000000000000000000000089
:105720000000000000000000000000000000000079
:105730000000000000000000000000000000000069
:105740000000000000000000000000000000000059
:105750000000000000000000000000000000000049
:105760000000000000000000000000000000000039
:105770000000000000000000000000000000000029
:105780000000000000000000000000000000000019
:105790000000000000000000000000000000000009
:1057A00000000000000000000000000000000000F9
:1057B00000000000000000000000000000000000E9
:1057C00000000000000000000000000000000000D9
:1057D00000000000000000000000000000000000C9
:1057E00000000000000000000000000000000000B9
:1057F00000000000000000000000000000000000A9
:105800000C0000000000000014B80000F87F000049
:10581000A3E20000883B0000000000000000000040
:105820000000000000000000000000000000000078
:105830000000000000000000000000000000000068
:105840000000000000000000000000000000000058
:105850000000000000000000000000000000000048
:105C00007B00000036000000460000004600000057
:105C10004400000042000000440000003400000086
:105C2000390000002D000000410000003800000095
:105C300039000000420000002D0000003400000088
:105C40003100000041000000430000002D00000072
:105C5000420000003100000033000000440000005A
:105C60002D00000043000000370000003600000057
:105C70004100000034000000340000004300000038
:105C80004400000044000000420000003100000019
:105C9000310000007D000000000000000000000056
:105CA00000000000000000000000000000000000F4
:105CB00000000000000000000000000000000000E4
:105CC00000000000000000000000000000000000D4
:105CD00000000000000000000000000000000000C4
:10600000FFD80000FFE00000001000004A4600003A
:1060100049460000000100000101000000140000DA
:106020000014000000000000FFDB0000004300003F
:10603000000600000405000006050000040600003C
:10604000060500000607000007060000080A000019
:10605000100A00000A090000090A0000140E0000DE
:106060000F0C000010170000141800001817000093
:1060700014160000161A00001D2500001F1A00004B
:106080001B2300001C160000162000002C2000001E
:1060900023260000272900002A290000191F0000DC
:1060A0002D3000002D280000302500002829000098
:1060B00028FF0000DB00000043010000070700008C
:1060C000070A0000080A0000130A00000A13000073
:1060D000281A0000161A00002828000028280000AE
:1060E0002828000028280000282800002828000070
:1060F0002828000028280000282800002828000060
:10610000282800002828000028280000282800004F
:10611000282800002828000028280000282800003F
:10612000282800002828000028280000282800002F
:10613000282800002828000028280000FFC00000B0
:106140000011000008000000AA000000FC0300008D
:1061500001220000000200001101000003110000F4
:1061600001FF0000C40000001C000000000100004E
:106170000501000001010000000000000000000017
:106180000000000000000000000000000602000007
:1061900003040000050700000100000008FF0000E4
:1061A000C40000004B1000000002000001020000CB
:1061B00004030000050500000407000006030000BA
:1061C00005090000000000000102000003040000B7
:1061D00011000000051200002106000031410000FE
:1061E000132200005161000071070000143200000A
:1061F0008191000042A10000B1C100001523000000
:106200003352000092D10000F00800002462000028
:1062100072820000A2160000B3E1000017430000E4
:10622000B2D20000F12500002728000044450000FC
:106230005373000093C20000FFC40000001A000066
:106240000100000002030000010100000000000046
:10625000000000000000000000000000000000003E
:106260000001000003000000020400000506000019
:10627000FFC4000000250000110000000202000021
:106280000202000002030000010000000301000000
:1062900000000000000000000000000001020000FB
:1062A000110300002112000031040000411300001E
:1062B00022320000510500001461000033FF00008D
:1062C000DA0000000C0300000100000002110000D1
:1062D00003110000003F000000C70000129D0000F5
:1062E000C26A00006EE0000002FB0000E1A80000AE
:1062F000E8E200000753000077AF0000BE2700006F
:10630000574E0000B18500000C6C00000EF8000034
:10631000874B000033D400005508000029DA000044
:1063200018C90000566D00007330000050340000A2
:106330008B9100007F1B000072180000D1620000EA
:10634000B63A0000A81000007740000003080000E3
:106350007A980000E2E40000E6E0000090400000CF
:10636000F4F10000FCB10000593500004545000083
:1063700044A4000033BB0000484D0000AF7B000088
:106380009B8C00003657000048420000194900006D
:106390006BF7000045EE0000BEB80000845100001D
:1063A0002C1A0000B7530000109600001B6A000072
:1063B000BB9E000076E800002DF90000E2340000EA
:1063C000B5520000B9D9000082DF0000CB08000000
:1063D0008A9A0000590E0000C0010000E27A000015
:1063E0006254000054000000AFEB00001C9F00004E
:1063F000F2EF0000881D00001152000073D8000069
:10640000C919000045720000F63700003CD70000B3
:10641000D309000058A400006F8500000FCB0000D6
:1064200016B10000D3C5000018EE0000A6FE000063
:10643000270E00008DB900000B7A00000C40000010
:1064400059540000B473000030E800003D710000B2
:10645000220A0000072C000054BA00008D620000E0
:10646000E6D800009A0E0000FBE100004A2F000071
:10647000CD800000B03C0000C5EF0000E43100001A
:106480000164000031410000182400001663000080
:10649000850A0000287A0000A93E0000B89100009B
:1064A000D39E00003D8800004B6300004B4D000070
:1064B0000A9000007B2B0000DBA50000F1DF00004C
:1064C00077850000493D000098030000C30F0000DD
:1064D000C48600004911000016D7000062000000C9
:1064E000B90300009F990000D86100006E90000081
:1064F000AC030000BE7D0000E75900000C800000E6
:10650000772D0000D0EA0000077D0000EFE50000D5
:10651000884B00001A5A0000489800000B980000B1
:10652000D6EA00004D88000027490000E839000045
:1065300075C600008B9F00007B3C0000393E0000C8
:10654000534700009DE500000BDB0000E5950000CF
:1065500034B100004F2A0000F392000002C0000096
:106560001B300000EA97000024820000395F000021
:106570007DAD0000802A000020030000B4EC000084
:106580000B08000086B000004ADC000003E20000B7
:106590006DE10000E7E500008FA5000092690000B2
:1065A00072E50000CBA0000081CA0000982800001E
:1065B000E188000083C90000BF560000A4DF00008E
:1065C000C7720000702300000F910000D229000064
:1065D000926E000007CD0000B9AC0000C6A100001B
:1065E000BDD6000032C400001D980000817200007A
:1065F0007CB1000065C000005C0B00002E7D000037
:10660000C630000065930000C124000070D3000074
:10661000CD7C0000C09E0000512200009BB800000D
:1066200027C70000623E000078D500000706000082
:1066300064C700008E7200009CE20000921400000B
:10664000832E0000ED5A00004ABA000023F000003B
:10665000C6E100004B2100004FF00000970A000047
:106660002DD20000FD460000F82C00009B310000F8
:10667000774A0000B10C000071C200006AE400001B
:10668000EDA7000065400000A6460000D2AB000068
:10669000DEFA00007D490000C5F10000F8F20000BC
:1066A0005AA200008F3C000068C20000BDAF00008D
:1066B000E41F0000A0FD0000A1E600005FA30000B1
:1066C0000FBB0000D25400002A4F0000069B0000C0
:1066D00081A10000D012000007CF000050C00000D0
:1066E000354C000075720000C1040000321000003B
:1066F000F1C000009A23000002D7000002E400006D
:10670000F3B60000FB9300008DD70000DB9500007E
:106710003C3500005C2F0000906600009FFC0000EC
:10672000D4320000BD13000011D500006DAD000093
:106730007E960000FBCE000031AD00002C6F000003
:10674000DD660000B5EF0000617B000058D8000056
:10675000FDF800000D530000E2320000137200004B
:10676000452300002B4600007BC1000097D30000AA
:106770000B4A000099530000E16B00008F3C0000C1
:106780005BB00000046F0000B8F30000E986000071
:10679000A7A300004B9E0000D23E0000CDBA00002F
:1067A0008B5A0000D8050000C8D10000E61D00008B
:1067B000245200003D0E00001E3E0000EF5200007B
:1067C00036B100003F7E000023CB000040CB00002C
:1067D000BC67000050F0000038880000CAD10000FB
:1067E0009EF20000918800004EC900007351000025
:1067F000326F000019D400003C090000C4420000C0
:1068000008B800002B63000087E900006B0C000053
:1068100052A70000697700008AE3000050060000DC
:10682000C6DD00006D8900005DAD00003D53000035
:1068300015D2000046FD0000D0DB00009C400000A7
:1068400095B80000F5BD00007EB800009B57000021
:10685000462300000A6900008B3A0000E917000097
:10686000D5CF000096200000DCDC00008B1B000070
:106870008E7E00005889000011330000BF5C0000CC
:106880002994000004530000AEEC00007E250000B7
:106890001B150000F9E10000A24E00001E8600005A
:1068A00009A60000074400004EC30000A900000034
:1068B000DBEB000088DA000041EC000045BC000082
:1068C000FEFC00007BE40000712D000032F90000A6
:1068D00049BC0000D247000010F000002DAC0000C1
:1068E000DBD000005F0B0000F7380000976E00005F
:1068F000D2460000B7500000B6180000A3C900003F
:1069000010F0000063550000DBCA0000A6F700008D
:10691000D8DE0000FEB800008E23000032F7000031
:10692000150B00007A8B0000FD7100006D35000032
:106930001DC20000F687000091E4000030E2000074
:10694000204B0000050000000C5A0000828A000065
:10695000E82800005D58000017720000A7A00000A2
:1069600006D60000C4E80000291100005AD100003A
:106970002DC90000F2DC0000FCFA0000E16E00000E
:106980002EBB000074C70000125200009DE50000FD
:106990002CA400007323000004A4000085AE0000B6
:1069A000C46D0000EA080000B0C20000E6970000D5
:1069B000B69A000049420000AA6B00003AAC000001
:1069C000BC850000F7DB0000EB860000A39100000F
:1069D00092400000EBCC00001BDF0000E2FA000058
:1069E000E39300004CB7000066760000504E0000B4
:1069F000E6DF0000CB100000A0AC00007B7F0000B1
:106A0000138800008F5F00000A8B0000292C000013
:106A10007C86000023BE0000647E0000C46000008D
:106A20007A9C000040D10000677C000076F80000EE
:106A3000A47A0000E9D80000ECFA00007D0600000E
:106A40001A790000E46D0000CC8C00007E76000016
:106A5000C425000017C50000D4730000603000009A
:106A600093340000639C000089F50000C52F0000EE
:106A7000652900009D610000D25A000056B0000058
:106A80000A0D0000C927000090C300004414000054
:106A900062AE0000BA5800001B10000045880000DC
:106AA000C40A000089790000EF300000DEDD00003C
:106AB000AA5F0000D4FE000058D000003D980000FE
:106AC0004BC1000099D400009FA00000B3FA000061
:106AD000023300000A8B00008A6A0000E4A800006C
:106AE00078F50000B7350000422F00006527000050
:106AF00096E00000838C0000919C0000B73D0000F0
:106B0000C81D000071770000C3B40000D20A000065
:106B10009F7A0000B81D00009EE80000EA6F0000A8
:106B2000A49000000DFC000035720000F317000077
:106B3000BE0300007489000028E80000DDF20000B8
:106B40009E0D0000A5E10000DE21000086BF0000D0
:106B50002BAB00009F4C00000EEA0000F4B50000D3
:106B6000512C00008B2A00001D9A0000363B0000CB
:106B7000742700007F110000E5820000391C00002E
:106B8000BC8C000074E900005249000058F5000078
:106B9000EA0A0000BBD8000061500000D4A6000043
:106BA0006F920000E5F90000D42400003AD60000FE
:106BB00020ED000080370000D13A00008B3A000041
:106BC0009FC70000E78A0000CCC2000053240000E9
:106BD00091D20000AB110000DA020000D2300000B8
:106BE0001BE800001FCF0000963600006250000036
:106BF00051E700001ECC000032E5000027C5000070
:106C00008A930000305D00006529000091EA0000D1
:106C10001D76000062A40000055F00009F2E0000AA
:106C20009EB8000040AB0000AABF00007A910000AF
:106C300034F300003A250000EF5B0000E988000013
:106C400092CD00003C3200003411000044230000CB
:106C50008D0E00009178000099EF0000B0E4000074
:106C600006DF00003F2C0000761A0000D94C00001F
:106C700081190000565600001BE90000552800004D
:106C8000E0780000E86200003EA00000E2AF0000F3
:106C90002CDF00004316000028C70000B179000077
:106CA000AD2D000007130000E54B000097570000D2
:106CB000B54400003D940000C2A20000C8000000DE
:106CC0007D5600002BD70000623B0000D88F0000EB
:106CD00099640000193600004FEC0000FF0000002E
:106CE00088A00000CA280000A457000034AA0000B1
:106CF000ED53000051200000790800000E960000BE
:106D000000800000028300006DC0000002E7000068
:106D1000C7080000A97A000089E600005688000034
:106D2000149600002208000058940000315B000017
:106D3000EF660000627A0000DF90000018AA0000F1
:106D4000F69D0000C5090000967000002252000068
:106D5000A153000098E700002A970000451B00009F
:106D600024200000866300007E7B0000B0B7000096
:106D7000858600002B3600009C6D0000F644000064
:106D80009A920000E264000096EE0000E1C200006A
:106D90001E6D00004C5B0000B4D30000A47700001F
:106DA0009B730000B6DB00007D31000056B9000087
:106DB0009A13000076880000A83F0000BA7A00000D
:106DC000E1F80000AAE30000665D00002D6300000A
:106DD000CC5C00006F8400001A690000928D0000F6
:106DE000D4D80000923C0000472C000079860000B7
:106DF000B1B8000004790000E3920000CCD200009A
:106E00003BC80000EECE0000C6EC0000CC0E000037
:106E1000EC7C00007F2C00004CA20000A0A8000029
:106E2000CC85000064B00000682F00000105000060
:106E3000906D0000A8920000C2E30000E98100000C
:106E4000292800002B6400004AFA00002AA4000050
:106E5000A28A000053B00000D07C00004621000050
:106E60004B4B00002A7C000020B00000E42D000005
:106E7000CF170000CD970000D73200008FEE000042
:106E800075160000F14400002DF800006257000064
:106E90000FD30000C0D50000F34B00005C81000060
:106EA0002381000004A1000025BD000089BE000070
:106EB000D707000098B60000153C0000D084000001
:106EC0005CAE0000CBA80000BBA200008F2A00002F
:106ED000A3CD00002AAA00000C3400009475000025
:106EE000152C00002D700000884D0000879F0000C9
:106EF00087AE00002D2B0000725A0000682D0000A4
:106F0000FA460000A512000071B90000829E000040
:106F1000CEC30000D4830000607E0000A7170000ED
:106F2000DC530000C5950000335E0000832E000096
:106F300041450000482E000008500000033F0000BB
:106F4000CFC30000EFC0000089240000DCD800009F
:106F50009BEF0000B9BD0000B19E00003967000042
:106F60003DBE0000862C000075D80000E5A9000099
:106F7000A03F0000DD690000956D0000F6A500004F
:106F8000EFB10000F3F00000FBAF0000E78E00005F
:106F900049330000C8420000C8EC00004730000040
:106FA0003A0F000096230000B3B200000208000070
:106FB000BB9E00004A310000E88000000FDE0000A8
:106FC00020C800007EEC00005C620000490F000059
:106FD0007A5A0000FE4300007C360000ECAA000054
:106FE00045EF00006B6D0000E98700000EC3000054
:106FF0000C340000134E0000C5A300008FBA00003F
:107000000E9100008AFA0000093E0000473200009D
:1070100035CF00004E4300001CC70000A7D1000080
:1070200016910000A86E00002E4E0000204B0000BC
:107030005963000068850000FCCE000036D90000CE
:107040009E8900005348000091C6000059C8000006
:107050001D3100000A4A0000E0AA00000C68000090
:10706000594900002BA800008F0C000057D50000E4
:107070004864000065D400004DCE0000F86E0000AA
:10708000FDDB000002740000FC5A00006FDD000010
:10709000DFF30000C004000089320000D64A00007F
:1070A000FC8E00009F4C0000304B00001DD80000FB
:1070B000DCF900009C2700000FD20000D3F600008E
:1070C000ECC400009B220000F3C400000218000082
:1070D000F96F0000E58F000062C20000A692000078
:1070E0002581000099360000B6F70000BE2200009E
:1070F000D2F600002FA80000CCDB000081F00000D9
:10710000E20500008CE30000A01D00003AAC000086
:107110006DCB00001CB50000BEB80000F1E8000017
:10712000371D000076380000843D00007DC7000058
:1071300096170000132A00005EF10000AB0B000060
:10714000116200004D810000F1DB0000AE12000072
:107150008A2E0000031B00000B6E000071ED000082
:1071600085C70000C58800004B1D000095FB00008E
:10717000778900006285000003AA000088C2000031
:10718000C63E000022360000FA9E000078D70000BC
:10719000FD9A0000F0960000539B00003351000060
:1071A00056670000060A0000A8540000158A000077
:1071B00038D400009A8B00007C5A0000598D0000E2
:1071C000B55E0000E48B00007863000030E1000051
:1071D0009A7E0000D3310000ED4F00002A750000B8
:1071E000D40F00008BF200005FC400009F960000E7
:1071F000351E00000FE3000069F800003237000080
:107200002D4B00004F53000097030000DAC9000027
:1072100003460000352F000042C80000DCC100001A
:10722000BFCB0000F1C20000E52D0000D1590000E5
:107230003BE80000D3E8000029E90000328C0000A0
:10724000B5F20000ECA6000007860000959800004B
:107250003CA60000572F000024AD00006E6C00001B
:107260004EC30000D0010000BE2B0000537C000084
:10727000D2B000009DD80000685B0000DAFD00007D
:107280002FF900009C5900005356000053E70000FE
:10729000340900009BE50000939A0000AA1A000040
:1072A0008EF10000936D00004AD70000F8650000E1
:1072B000039300008EA3000015B100008FFD0000B5
:1072C000A15D00007DEE0000CBFF0000008000000B
:1072D000637C0000B8FC00007F530000163B0000F8
:1072E000E7B10000EA6A000049EB0000F534000055
:1072F000730A000068120000429700000A1900009B
:10730000DEC40000DEC40000DC0E0000BD0F000083
:107310002C27000034CB0000BDDE000024920000CA
:1073200043EF000034E50000C0600000EA350000D3
:1073300021260000D70C00002C6D0000F2BF0000D9
:107340009E2400006539000084540000BFDC00006A
:10735000A72500001CBB0000346C0000DB2B0000E4
:1073600002490000BDF900006E4900001E3800000F
:107370006EB3000032F70000DA1300004FFA00008D
:1073800097A9000095EC0000FD9400009AD600003B
:10739000350D00006BEA0000E87400008B5B000014
:1073A000CF0A000054910000B3430000597E000052
:1073B0005925000055330000C8260000F75A000088
:1073C000724800008BB3000055270000AEED0000AE
:1073D000706F00007E7B00005B9E0000F7C4000021
:1073E0002CEB000027CB00006A28000024CA000014
:1073F000F88D0000167A0000684900009E29000000
:107400008B040000642C000077D20000C3E1000070
:107410003716000022D60000B5BD0000059500001B
:107420000E6B0000051E00005ED40000B2CB000011
:107430001A55000043DD000045950000AC1A00001D
:10744000E6C8000049E800000DAD0000F2C00000F1
:107450005719000071DB0000506600006B1C000033
:107460005449000050EB00000E86000077620000D7
:1074700063240000905B00004EDD0000E036000059
:107480001F3C00001B4900006C92000085AD00000D
:107490001957000019D10000E4F40000D980000061
:1074A0008B870000E0AD00008E080000AF190000DF
:1074B0007A9700000FAF0000C2C60000C2C20000F1
:1074C000F7C00000FC8800006376000056E9000069
:1074D0006E580000BCCE0000EAA20000ADCC000057
:1074E000DE4A00006A6100004C84000096780000CB
:1074F000D58900001ABC00004786000020E6000085
:107500009BC500004C480000B31400003BF900008C
:107510005F190000164500006C6F0000071A00009C
:10752000B23D00001AD500004D3A00004548000069
:10753000AF240000AFC9000016F800002D8E000037
:107540001196000044C80000D20900006B5D0000E5
:1075500074CA0000CA7B000088080000074D0000C4
:1075600087C4000070BC0000B28D0000F29A0000D9
:107570003860000081180000E695000042F200002B
:1075800095BE0000A4070000922800001CAF000078
:107590008BEA00006E040000CF9D00000354000041
:1075A000C11D00001EAE000042A10000ECD600008C
:1075B000E7F000000DC70000CED80000C39B00001C
:1075C0002BCA0000E97400003F1C000012DB000021
:1075D00005D0000018EE0000632500006DB9000022
:1075E0002A7F00002C750000DE490000459D000048
:1075F0008B8F0000337F0000FD3E0000FC1B00006D
:10760000D3FB00003CA8000022F3000057C4000098
:107610000F820000C45B0000F1C30000155C000095
:107620000198000022160000A7A80000A6980000FC
:107630000E8D0000753F00009E150000F13F000018
:1076400043AE000020640000B1A40000AA56000070
:10765000400800001D3100000E7A0000595500005E
:107660000FBB000038BF000040E70000962E00006E
:10767000B31C0000B2B700002C6D000015F4000030
:10768000F2450000BF3200002EA70000C2C4000077
:10769000621F00002DF0000039CA000004D3000072
:1076A00007D50000246900001948000070DF0000C1
:1076B000689E00007F2C00004D80000015520000E5
:1076C00008550000F4370000BFAE0000274F00004F
:1076D0001099000036D9000087230000E0710000F7
:1076E0005F240000BD8C00008C8E00008C640000C4
:1076F0005F0E0000B8D300008F2A000090B9000090
:107700002E2300008E2E000000DE0000DD6D000044
:10771000CED80000954F000099510000056B000085
:10772000971700003700000025EC00002C2C00000B
:10773000315C0000677200007645000003FC000029
:1077400047F90000622A000049D8000020420000EA
:107750008DE30000B72C000031F4000029C90000BF
:10776000338F000021960000DA8D0000C9F100007F
:107770003B0C000020730000F218000073B0000002
:10778000900B0000315100007E600000B75C0000EB
:1077900026780000A48E000032C0000003B700006D
:1077A00030710000A85D000090CB00006A940000DA
:1077B0009E8300001DBE000038CA00006208000061
:1077C00058A900000EBA00008588000024030000BC
:1077D000E58E00006A1E000023130000655E0000B5
:1077E000CEDF0000C0EF0000899400000CD1000043
:1077F0004551000028890000E48D00006C5800000D
:107800008E4A00000EC3000010FD000030A80000EA
:10781000A3920000691600002815000099DB000003
:10782000EC8B000093FF000000510000E7D3000044
:1078300010820000EA2A00005A770000249200001B
:10784000A9E0000030CE0000DEBE0000A312000060
:107850006AA800002AE80000D41A00009A79000003
:107860002307000091610000B1C400006C420000D9
:107870001DD500008F6A0000C73C0000ED8E00009F
:107880006A18000084150000AB1E000026C000002E
:107890009C27000050C7000045D9000082A00000CE
:1078A000BB13000061EB000088400000BF860000B1
:1078B00069CC0000597A00003DBB0000D3390000BC
:1078C0007B780000817500005FC50000BEB8000035
:1078D000B26C0000ADB30000EACA00005CA2000078
:1078E0001ACA00003A4F0000786B0000B4D50000BF
:1078F00053080000915000001E640000922E00000A
:1079000049B60000C30E0000474E0000B4C8000096
:1079100090230000029100002AC70000E9610000E6
:10792000BFFB0000B57D0000701F0000C5530000C4
:107930002CB9000096860000F863000050B60000E5
:10794000BF2D0000AFF900008C230000F5200000DF
:107950003FF800007D250000C33C00003596000084
:10796000F01600004F57000049960000CF2D000090
:107970005545000042860000A9AD000071A5000039
:107980005D54000072450000160100003C0E00002E
:10799000F7C3000011480000F1D40000BCF3000060
:1079A000AAC700001CF60000283A00008B0B00005C
:1079B0005DB100008EFB000030CF00003896000063
:1079C000A33000008B87000072A600004ACA0000A6
:1079D0006A9B000087820000A01700008E0500004F
:1079E000FB4F0000B6EA000000B90000362300009B
:1079F000D0E3000041E300006CE70000F455000014
:107A000034910000CEC00000C509000053DA000028
:107A1000C7DE000077D500007D2000000E84000046
:107A20008E7B0000DB1B0000797D0000290900002F
:107A30008C2A000076C2000039A100002CED000065
:107A40002255000085560000EF69000090060000F6
:107A50004DFD000079610000B35500001D350000A8
:107A6000398E0000398C0000AE6F0000A4B0000019
:107A7000000F00005B740000C6500000BC6F0000E7
:107A80001ABB00007BBC0000733400008D160000A0
:107A9000CA6F000021ED00002FF000009B90000055
:107AA0003E7F0000761C0000938F00003B19000011
:107AB0006F3C00004EAA0000CE960000EE8600004B
:107AC000256D0000DEB80000D5E3000085730000DE
:107AD000469F000082750000668500002D72000040
:107AE000D44B00000B97000068A70000688A0000D4
:107AF000CBA400000D4A0000548E000060F8000086
:107B0000DCEF0000E78A00000E290000CAFF000039
:107B1000004A0000D0D500000A000000F2BC0000BE
:107B200072340000D1A3000001AC0000D82D000089
:107B3000F7F3000007910000BEE300006B60000057
:107B40004A7E00003A610000190B00004D29000038
:107B5000043A0000DD8200008D56000061A700009D
:107B6000A0BF0000779E0000FCED00006DB000009B
:107B7000DC3C000043EF0000B9940000B4F90000C1
:107B800077BC0000E5EF000026D00000CB0C000021
:107B9000863D0000561B00002BAD0000EDE5000007
:107BA00071E30000BE07000035EC00001F1C000060
:107BB000C15D0000CC8E0000C6E0000006E70000BA
:107BC0006F960000E7F20000C6A10000C11C000093
:107BD0001FEF00009C3C0000D9B20000F60D000031
:107BE00054650000EC21000085D0000016D500008F
:107BF000CC110000D2F70000279F0000873C000056
:107C000051FB000026E00000D7E30000DE2C00005E
:107C100014520000BBA500001C570000A8AB0000D8
:107C200096DD0000ED170000E9E000005B55000064
:107C3000BCB90000E3E90000F8F20000BCA70000B6
:107C400028A400004CBF000027A00000A58200006F
:107C50008E2D0000B50400000CCE0000770400005B
:107C6000DCFC0000FCF100008E5E00003CB2000075
:107C7000EA2E000083390000D766000071930000EF
:107C8000E44F0000C3080000F14500003534000057
:107C9000B9BC0000A08A00008AF400000D2B00008F
:107CA000A5C70000C1190000B8B0000000730000B3
:107CB000B5AF0000F74F000017DB000053B4000021
:107CC00084F300002C6E000049F10000F3C50000B1
:107CD0009F100000E5510000D1C40000D5D4000081
:107CE00060C6000010DE0000686F0000DC230000AA
:107CF000A91E000016E700006C54000096B20000B8
:107D0000DC020000CDD0000028B900006DEC0000BE
:107D100000F30000DF160000960700008A930000C1
:107D2000198F0000229400005B1B0000A980000056
:107D3000542A0000B077000046530000DC740000B5
:107D40003CB00000D15A0000E4D800003D3C0000E7
:107D5000D6F100005D270000D6E30000AFD300009D
:107D600004B400009C3B0000AC160000CC65000091
:107D700090B100003BC300001B10000000E70000B2
:107D8000BB5E0000E4FA000011870000AA38000082
:107D90006E8D0000D2D40000F24F0000048300007A
:107DA00093AB0000B37F0000B49200003EEB0000F4
:107DB000F9E10000CBC600009356000051E7000037
:107DC0008A600000E4B1000025440000463A00004B
:107DD000945600000C2C0000CA7700001F7E0000A3
:107DE00033CE00002EE00000D1480000AD5B000063
:107DF0009406000030F30000920B0000DCA70000A6
:107E00009AF90000791F00009634000079630000A1
:107E10009A9A0000A5E900006A950000448A0000D3
:107E2000030200009BAB000029E4000041EB0000CE
:107E3000E78F00005FEA0000719E000078E9000013
:107E4000D487000046560000AD1800000837000037
:107E5000008E000056BF00002B1F00002FBF000047
:107E60000C550000D32C0000EAA5000058070000C4
:107E70005E440000F2C10000671E000064CB0000F9
:107E800095E60000A26A000075D300004B53000085
:107E9000DE500000392B0000F5510000E5E1000044
:107EA000E7810000A22E000008F10000F0C60000EB
:107EB0004770000096860000FE950000334E0000DB
:107EC000CABD0000887B0000C4140000D515000066
:107ED000DC4700004F1C0000550A00008C9A00008F
:107EE000213700003A850000C6E400008BEF000057
:107EF000B60A000020FE0000CF790000598C000077
:107F000019730000BAF600006F140000550300005A
:107F1000E96C0000679C00003BED00003EA70000FC
:107F200027A3000086950000FB0300003C0300002F
:107F3000B3120000C9BB0000E9B700002B9D000090
:107F4000FC390000608500003DB50000E61A000025
:107F5000458D0000311E000026FF000000CF00000C
:107F6000193300002F2E00004EE2000063FC0000D9
:107F7000B6990000936700006B010000AC7600002A
:107F800085D50000D1BB0000C48F00001C57000045
:107F9000089000008DAE00007E7B000062040000AF
:107FA000D29200007BDB0000FA6D000089740000B3
:107FB0001ABB00002248000023BD0000B0C700002B
:107FC000A3B0000051120000B6800000C779000085
:107FD000231D0000CFB40000A4E2000021950000A2
:107FE0000D32000022C60000BDA20000B1660000F4
:107FF000905E0000ED70000005AD00007F2C0000D9
:108000005CD60000D42C0000313800000C0B0000BE
:1080100091B000003E3E000078A50000EFD50000C2
:1080200054DC00002832000048DB0000002C000077
:108030002E760000C405000012320000EA1A00008B
:108040008CC60000A3B00000A60000009B5C0000EE
:10805000B1E40000BEB8000038C90000B2AA0000B8
:108060007C8A0000069E0000AE55000032B600007B
:10807000DA870000D9F200005C700000C916000029
:10808000414E0000B494000090800000CE810000BA
:10809000849D000049DE0000F7FA00000FAE0000EA
:1080A0002927000092590000A52D0000348500000A
:1080B00080DE0000C4ED00007FCB000010940000C3
:1080C00011BD0000665900009A9100004D3000007B
:1080D000717E00004CE20000DFFA0000E0270000A3
:1080E00038A000005A5A0000893400009360000054
:1080F000D660000005FD0000316F0000959800007B
:10810000EA3300003822000004B2000083AC000013
:108110009B5E0000C00C000043E2000009BB0000B1
:1081200059670000280F0000EB2400002028000001
:10813000EB63000082460000B653000054080000C4
:1081400004ED0000EEAD000029870000EC9900006E
:1081500000530000CBAD00008FE10000F3C300002E
:108160005BE300008D7500003660000041F0000008
:1081700022D80000E7CF000015210000DFAE00008C
:108180002EB800004A9A00003AAC0000DA32000033
:10819000FAC70000620D000042DB00009773000088
:1081A0007B1F00005B6200009598000028B900006A
:1081B0003738000027E00000643A0000331A00005E
:1081C0008B5A0000C91C000023FD00006C5B0000FE
:1081D000F04300008ACD0000D2B0000030860000DD
:1081E00021A6000020490000B6D700003E7B000019
:1081F0000C670000B5B300001A9A0000B9660000D1
:108200003F6D0000C9060000D7FE0000BA60000004
:10821000F3340000729900007CC400001B120000BF
:10822000A5470000D3000000F25300004890000072
:1082300000F200002E910000BF2F00004C570000FC
:1082400012ED0000910C0000D34F0000352C00000F
:10825000A24A000059650000864F0000B2F10000FC
:10826000B90C00003D2D0000F81C000014E40000D3
:108270009C4100001CD4000095710000F11D00001D
:1082800054B5000088CE0000922A00004C1A00006D
:10829000472C00003AEA000037F00000E5810000BA
:1082A000568E0000EBF100008F9A0000138D000045
:1082B00093D800003F03000052660000A2AB00000C
:1082C0003ACE0000A9520000AA9100000F650000FC
:1082D0004D140000ABDD00002D7D0000D88F0000A4
:1082E0001E9F00005C3900002B6100006D2D000016
:1082F00090B20000987200007CD40000BD560000CF
:10830000574300000CC60000E55A0000D0D800001A
:10831000A162000008D80000B1020000D6B700003A
:108320002E580000215C0000B29A000058C30000E3
:108330004D4E0000BAD8000030D20000005B0000B3
:108340006A3A0000882100006C3700003FCB000033
:10835000960A000033FE00001DC90000BF4900005E
:108360000A6C0000A32C0000A3A20000952F0000BF
:10837000DAD4000053C60000508D0000AE14000097
:108380005AD7000006FB0000EDE30000E07100009A
:108390005D2E000047530000123300007BC8000030
:1083A00008050000F51200000F2F00002D37000017
:1083B000FBF10000678A000085CB0000C9F40000D3
:1083C000D83100009F7600003975000004B300002A
:1083D000B05300000C6A0000EB1A000033310000BB
:1083E0002C480000BB01000072460000FE36000071
:1083F000DB190000D6650000C53E0000F551000005
:108400003D4D0000365E000090D700004EA50000F4
:108410001AA00000B9660000008F0000B3B0000091
:1084200002E300006C6C0000353E0000CCA40000AC
:10843000CDA80000A6A80000FD210000354D0000D9
:1084400078420000860A0000870800008848000083
:108450000400000040E50000B8F50000E58C0000D5
:1084600077390000C9060000459B0000C94D000097
:108470009A510000344E0000BDD300000B92000062
:10848000D6EE0000937000007A830000F7610000D0
:1084900053B80000FA2F000009370000A4CD0000F7
:1084A00087FB00002ED40000CF4D0000C3FC00006D
:1084B0006F3E0000590C000075390000B2A40000A6
:1084C0004F140000523900005ED3000069360000EE
:1084D000BFAD0000FEEC00006C1400006D33000026
:1084E000D34300002552000008A7000064060000E6
:1084F00055060000FA1800008DC60000AEA200006C
:10850000F7C70000CCDE0000C7A90000A6CC000021
:10851000B8DA00001A6A00005EC20000984F00003E
:1085200004BA00009150000000C00000293600008D
:1085300027D60000D8320000CE620000CC32000006
:10854000ACC600007A69000066AC0000578D0000E0
:10855000B92C0000CED70000BFF9000048BF0000D2
:10856000E38A0000E3F2000063090000716B000081
:10857000B0CB000013910000B1660000A51300000D
:108580002BAB0000351B0000C7D900003EAB00003C
:10859000F22B0000A4DF0000031C00003285000065
:1085A000F33C0000AD66000006E00000EBFF0000B9
:1085B000005A0000C64F0000FE2B00001C05000002
:1085C000E5940000B5730000544300002E670000DE
:1085D00051500000B112000019620000798B0000B8
:1085E000B4840000F22C00000120000001E1000032
:1085F000F5C100003D5400006EF00000908E0000B8
:10860000D1CA00000DD5000081B100000C0F0000A0
:108610002F4E000078190000734600004EE800005D
:10862000BC31000034820000E83300008A79000089
:10863000B3BA0000BCA90000239D000067A700009A
:1086400045900000B3440000446C0000A4F2000018
:10865000563B00006DCF0000163700001E4700009B
:1086600018360000606400008EB10000E3A800002E
:10867000926E0000D46F0000691D0000891B00008D
:10868000F42700009E1B00008EA60000782C00003E
:1086900063A900009E1D0000F9AC0000CE9600000A
:1086A000FA720000C3630000E5240000AA85000000
:1086B000BF1C0000D7B80000BE350000D145000047
:1086C000283A00009D65000029710000CB49000098
:1086D0001D3E00006A0E000029390000F5B70000B9
:1086E0009E070000786E00005CCE0000B4AC000075
:1086F000B57500007552000050C600002F1A00002A
:10870000CCFA0000B51B0000581100007DCD000020
:10871000B7FA0000E0880000F2C600007CB3000059
:108720005376000068C7000017180000D307000048
:1087300038FA00008D6B0000386E0000A182000046
:10874000FEB200009C89000050F800005BE20000CF
:10875000FF00000069380000C9460000FF0000006B
:108760009E3700002CDA0000312E00005758000020
:108770008DF00000B44C00003EE300008C2D0000A2
:108780007E050000279F00003FE70000F7E30000A0
:108790001E6400003A070000619200003863000088
:1087A000A9960000540400008B310000040D000065
:1087B000EE05000086290000A56E0000DA420000E8
:1087C000F2BB0000AB1E000089B00000030E0000E9
:1087D000D74D0000AA690000215F000085740000E9
:1087E00096230000C6D8000060720000C36200003B
:1087F000EA2900000A9A0000B63C0000B4B100006B
:1088000025D80000007D00004E200000CB3C000079
:10881000F3C50000335300005960000086DA000001
:10882000896100007DF6000016BE000021BD000039
:108830005CEC00009A1A0000425700000CEF0000A8
:10884000E7B6000037890000B3A60000E5AF0000DE
:10885000B9630000D4E20000D78500006113000076
:10886000E7B40000A08E0000EA3100007FA0000005
:10887000BE2A000070690000C07900007811000075
:10888000C95C0000C2C40000FEAE000031FB000065
:10889000A3AE0000022A000058710000510600003B
:1088A0005A5B0000D8490000DE270000D3FA000020
:1088B000381F0000AA6D000034F2000011D0000043
:1088C00062EB00008920000078E500008AA3000028
:1088D000BCFA0000C10C0000D6D800007F57000091
:1088E000C0FD000078760000802A0000217D000095
:1088F00046F700001BE20000CC3100007A270000A0
:10890000F0D6000098720000CCCA0000655100004B
:10891000AF6500000DEB00008A0C0000D25D000086
:10892000532000005BDD000045EE00003C700000BD
:1089300049930000534F00001F0D0000CD2400009C
:1089400091480000AB3B00008ECD00009814000061
:1089500006D60000BD890000DBA10000C574000040
:108960005954000053660000310C0000C1CA0000D9
:1089700041310000D0640000400A0000A92200003C
:10898000CA6E000036E70000D3AE00002AE4000003
:10899000913B000065070000C4E400001B96000046
:1089A000F1EB000085480000851C00006B5B0000B7
:1089B000122F0000622D0000B7F4000071A2000029
:1089C000F0DF0000B32C0000CB300000E218000004
:1089D000295A000036340000AD28000012CA0000F9
:1089E0001587000066A700007B910000CC6D000099
:1089F00088FE0000D1F200002A7C0000A25A00008C
:108A0000A96A00005DA30000ADA8000072F000009C
:108A1000D32E0000FD9C00007C860000BF0D0000EE
:108A200080B000001D300000148500007C8B000029
:108A3000971300003C1D0000E90B0000000000003F
:108A400018390000E15800004439000002B000006D
:108A50001DE90000EA1800009F480000D540000012
:108A6000FF00000098DF00004C030000C634000047
:108A7000A9BF00002FEB0000F963000041C900000E
:108A80001746000051420000A5AF000068C9000071
:108A9000D3E600005DCF0000E04600001593000023
:108AA000AA180000C85C00005750000060CB00000E
:108AB00092C60000C5E500000BF800009FCB000047
:108AC00014CA00005668000056FB0000861F000014
:108AD0004C4D0000E3560000FD5D00002C5E0000E0
:108AE000258F0000D2DF0000CF150000195B0000C9
:108AF000EB800000AB730000536C00005F100000BF
:108B00003D12000068B20000F7AE0000CCA90000E2
:108B1000E8680000FB460000A89D0000D634000075
:108B200045F1000026C20000FF0000005C7D00004F
:108B30006191000051C30000C3FC000039450000F2
:108B400093E50000ACAD000034230000B0560000F7
:108B5000E85C00007C4E00007E660000FE5C0000C9
:108B60008EF80000C97D000082700000C7BC0000C4
:108B7000E735000079FD000042FE0000AA980000E1
:108B8000767000005C6C000064220000CC7E000067
:108B9000400F0000AE3600000E1A0000559B00008A
:108BA000DF27000076D50000399E00004014000049
:108BB000F2440000D7710000F50400001F9E000081
:108BC000366300008FB10000537E00008A780000F9
:108BD00011450000454100004BE900000FD900009D
:108BE000296E0000765F00001F9800006F9900005A
:108BF000C2D90000054500005535000038F80000D6
:108C000066910000438F0000F00E0000F30F00009B
:108C1000985C0000554100005FAA00009E9F000084
:108C200047FD0000EAF6000087D50000B7FE00000F
:108C300078B10000A0A9000064AF0000A66F00009A
:108C40008A6300001BAC000042DF0000139D00009F
:108C5000205F0000F88E00002D7B000030A800008F
:108C6000B94C000023A30000327E00009CAD000040
:108C7000ECB40000FBBD0000943B00000E7D000042
:108C8000A01F0000081E00004A140000FCF10000B4
:108C9000937F000068EA000058940000649500008B
:108CA0004AB600009E4300002C2C00006DB9000065
:108CB00055D20000DF990000FAE3000064A2000032
:108CC00088510000D222000096D50000A06A000062
:108CD00077FD0000E2790000B7A90000DCFA00008F
:108CE0007CB100008A7B00007B990000E7A70000B0
:108CF000C924000062740000BBCC0000D1AF0000AA
:108D0000EEA0000008170000EBCF0000E785000090
:108D100066FC0000337E00002FD20000063D0000FC
:108D20008A550000AD270000B4BC00009D9E0000E5
:108D3000C04800005E0D0000FA6A00004600000016
:108D40007D4A0000E3710000E258000087E900005E
:108D5000AAA600009101000024860000F86F000020
:108D6000D0630000E5FC0000B6AE00004A0C000035
:108D7000C6960000B69A0000E26A0000795600002C
:108D800054B700005652000008FC000031F4000007
:108D9000B7110000E7B4000095D900001D3F0000A6
:108DA00012C1000026AA000026A200003513000010
:108DB00004F8000085890000B8F900001057000091
:108DC0001C8900005F340000CDA90000EC84000085
:108DD000EB2C0000664E0000C4460000CCFA0000F8
:108DE0006ED20000372B00000B6C00003AE100004F
:108DF000C8110000D1020000CAC10000DFC5000098
:108E0000469000007E580000CD68000078E7000022
:108E100036AF000097B500008787000033290000B7
:108E2000A99A000091A40000558A0000F1000000FA
:108E3000C2FD0000ED420000FA960000D6EB0000F3
:108E4000D3160000C73F0000CE23000058CD00001D
:108E50004F080000E6A8000028A30000D7990000F2
:108E600014A90000B82000008D990000013B00000B
:108E7000FC2400009C69000058DB0000459B0000BA
:108E8000A0AB000031CB000020CC00000AB40000F1
:108E9000AAC10000D45900005C0B0000B01800000B
:108EA000AD1C000033060000B532000048CF0000C2
:108EB00018370000D2C90000CF020000553E000064
:108EC000D2E00000A133000047530000459A0000A3
:108ED00053550000C7280000FD5D00004A2B00002C
:108EE000010900003B1D0000802A00006DCB00003E
:108EF00098C100003F0C0000718E000051C40000BA
:108F0000134900004F47000030590000A30700003C
:108F1000B8C000008D4A000005EE0000B7E900006F
:108F2000E37F000096040000A2E20000451B000061
:108F3000F41200002AAA0000A2AA00008B00000080
:108F40002C050000F6FA000063BF00002BE30000D0
:108F50008AC10000D752000090C00000F81C000039
:108F600077D40000DBCF00001409000003390000B3
:108F70004AA60000A19C000051E8000091CC00002E
:108F80006CA100001B9B0000123C00007F2B000026
:108F90007CF10000864C0000E20800005CC8000084
:108FA00008D10000B6910000F87D000071B9000002
:108FB000E6790000B51600005B480000D5150000FA
:108FC00073C60000AAB70000B0D50000BB1F0000A8
:108FD000018C0000033A0000A97A0000C9A4000037
:108FE00072BA00001659000059B400008F33000017
:108FF0007FC30000F0C5000025060000C89D0000EA
:1090000010A200002CC00000C8C30000BEE7000092
:10901000511E0000671D00002CA00000EE4500005E
:10902000F1E6000025570000BBBD0000BC71000048
:10903000049B0000B31D0000DBCC00007A6200003E
:10904000D48A0000376400004B0B0000614C000024
:1090500085150000091B000037C30000D709000078
:10906000C29D000092C80000157900000EF60000B5
:10907000FF00000011B90000C6CA000066760000BB
:10908000271A000047090000CD100000E1D80000B9
:109090003B320000ACD1000086D4000001DE0000AD
:1090A000F7370000C6700000AACC00007BA80000C3
:1090B000C47D000030450000C1C60000B3DE0000E2
:1090C000244A000059230000EDEC00001960000064
:1090D00066200000CA7A00008079000013E50000D5
:1090E000CF110000304A0000A8D00000485700000F
:1090F0004DC10000D04700002B5F00000C54000061
:109100002AC300004D2B000044AA0000A554000013
:1091100091B000001D310000453E00007B2400009E
:1091200031F6000030C000006295000036EF00000C
:109130009E470000AE3900003E780000D265000076
:1091400086220000AC6A0000596C00004DB6000099
:10915000B1C50000ED15000049B5000068370000FA
:10916000C8B200006A2E000024E10000EA330000CB
:10917000994A0000EAC9000012C400008AAD00004C
:10918000A3650000037200000F3B0000924900003D
:10919000F338000020E10000FF00000066740000CA
:1091A000F3540000F69900004B030000A05C00009F
:1091B000C33000002D1C000083A8000061B0000037
:1091C00017F10000E98C00006E960000AEA20000CE
:1091D0005CB200007CB600009E7500003D9B000064
:1091E0001A880000E1D200002E79000083F200000E
:1091F000FF000000A6D8000031E00000AE380000FB
:10920000E20C0000872B000035460000A8D40000C7
:1092100052C70000A5690000A0300000A969000045
:109220001CEC000003100000370300009F890000C1
:1092300022D800005DAB0000A26400005271000063
:10924000D1F40000D56C0000D0700000BF0E00000B
:1092500076F00000512C0000AD0C00004A850000A3
:109260006305000089550000F3E600004017000088
:109270001BFC0000F6C70000C5FE0000D133000053
:1092800038F30000DE200000CC2A0000699E0000B8
:10929000637900005A420000B39B0000B94B000004
:1092A000F3F30000E80F000090C70000D135000084
:1092B000FC640000F9C700000AC500005128000046
:1092C00045A90000A85100004ED40000E5080000A8
:1092D00061AB0000E3D400001B7B00001D210000F7
:1092E0006E3900005F14000073640000596E0000C6
:1092F00073970000C6950000948B0000215E00006B
:10930000EAB8000040AC00000F2B0000ADB7000031
:10931000DFA7000088C50000D2FE000009C50000DC
:109320000F720000ECF900009A3B0000F6620000AA
:10933000DD710000A16500008BFD0000C21500007A
:109340001C840000315F0000F814000062C30000BC
:109350003CF60000512500003BB30000E5B50000DD
:10936000AA690000FA7B0000C2DC0000A75D0000D3
:10937000D85C000091F20000DBAE0000153E00005A
:1093800049980000E574000042590000E8E400003C
:1093900096040000503B0000780700006ABB000004
:1093A000002F000075BD0000B9750000B615000063
:1093B00034DF000048D00000E48000009E30000050
:1093C000903600006112000093700000B1DF0000D1
:1093D000EAC70000F96200002F0B000050540000A3
:1093E00066990000C4790000751A0000B3D400002B
:1093F000543E0000850000005CF900009F41000021
:1094000087330000931D00006E600000D209000049
:10941000C4760000010A00003A1000006E07000048
:10942000A7AE0000371F0000603C000014320000AF
:10943000DA09000038860000B97F0000BCD50000C2
:1094400082290000B6200000A46400000BB60000D2
:10945000FD5A0000D8BE000018B60000C12600006A
:10946000923400008C9B00002EA40000E16E0000EE
:10947000178A000096370000548200008E16000004
:1094800067730000CAE3000076630000F3BF0000CA
:10949000D71000006AD80000D2650000D7A30000F2
:1094A00007B700008A8D0000927D0000FBAA000033
:1094B00074DC00005CFE0000F0240000D87800009E
:1094C0001F4C00000B7B000062CF0000DE4A000052
:1094D0008A2E000018A00000934C0000F5920000B6
:1094E000A1A90000237D000011DC000000BF0000E6
:1094F0003E67000006590000AA4500004FC3000067
:10950000D04100000A840000591A000035E700002D
:1095100063B9000004930000E7B60000E7C3000051
:109520001AE300002BB400002256000095830000CF
:10953000D0650000C2360000524D00009139000095
:109540005B9F0000962F00003876000082390000F3
:10955000E61900008328000011C60000A63A0000AA
:1095600070790000017B0000330F00005B010000F8
:10957000E80700008E210000C34E0000F9850000BE
:1095800050A400008D8A000028070000B67100007A
:10959000B68000004DEC00003D7C00003A730000F6
:1095A000C13500004CB10000D15100008D08000011
:1095B00000000000471C00006BFE0000D503000007
:1095C000EEBF0000860A000042310000C5DF000047
:1095D00021AC0000C49A0000BA840000A15200002F
:1095E00074300000D7390000F05E00005A7D0000A2
:1095F000491F0000407100008C7F00006899000046
:10960000AF9B0000E4F000005EC1000029DD000017
:10961000C81E0000259400007FFC00009C6C000028
:10962000395A0000CB490000593C00001564000085
:1096300049340000C3DE00000CA30000E40A00006F
:109640009F4E000043C80000791C0000619E00008E
:10965000DFA70000ED380000E6280000BA43000054
:1096600046890000F3D40000EDF8000030C200008D
:109670007C8700005036000061FD000099C40000A6
:109680004BDA000048AB0000B5890000037C000005
:1096900013F00000271800007E890000AFAA000028
:1096A000A1CC0000CF69000091D60000EA8A00003A
:1096B000657500002EA800000D860000AD3E00007C
:1096C0001B00000040B700002DB60000DB030000C7
:1096D000511100001B3B00001BD90000158E00003B
:1096E000C6DB0000DB0D000089720000DDB4000065
:1096F000D2D5000013CC0000FEB50000483F0000AA
:10970000EDF10000C6180000A4E20000ECD100005A
:10971000274F000047D20000028100000D3C0000EE
:109720004AF20000A5450000198E0000D034000068
:10973000750D0000244F000016D6000020580000D0
:109740000F2B00006F6C000071A80000695800002A
:1097500096EC0000103300000B1600004162000080
:10976000C3FA000038190000F64D000090E7000031
:10977000A32E0000796600009A6A00003CA6000053
:1097800041780000296A000048940000EAEA0000DD
:10979000E01000000A830000F5F40000E7830000F9
:1097A00059320000ECC600001B960000863900000C
:1097B000874300001496000027E40000D61F000035
:1097C0007E3300007FB5000008B700001B0C0000CE
:1097D00066BD000095B20000512300003543000033
:1097E00091140000ED5100001763000027BC000039
:1097F000AF6A00001D3C0000093B00008E670000BE
:1098000091F9000060400000F09600004B45000018
:109810005B930000D5E50000110C0000AEB600001F
:109820008A4000006A1C0000D46B000059570000F9
:10983000ED0300007DF500007DC300000728000057
:10984000956E0000C552000082720000C3980000AF
:10985000D71F0000FE6C00002865000095920000F4
:1098600030B600005A010000E7770000745B00008A
:109870007F09000038B30000F2A1000054D90000B5
:109880006E5F0000F4850000959B0000518600008B
:10989000208400002CC5000001E80000B73600005D
:1098A000DBC20000D6370000C577000016F10000CB
:1098B0001D3E00004146000075320000C9580000FE
:1098C000D7580000A0BE0000EDB7000033E500004F
:1098D00082A80000324A0000D9480000F7A9000021
:1098E000E38100004F31000008D40000DF53000086
:1098F0006FC30000007E0000D7F800003A0A0000A5
:109900007CBE00003CEB00002ED600001A1B0000BD
:109910002D40000067D400001C1D0000B5F80000B9
:10992000730000007CEF000084AF00002F1B0000DC
:109930009A8900001E54000064B500000E6A000001
:109940006AE50000A89C0000ABCB000023160000D5
:109950002D6E0000BD480000FC31000006A0000094
:10996000969F00004F54000016F90000FF00000011
:109970004313000006C20000F88000000EA700009C
:1099800076F10000361F000097DC000031AD0000CA
:10999000BD060000CF3A00006B220000E7BB0000CC
:1099A000E18E000084500000360300000AC200006F
:1099B0004DC90000BDB100005F640000203A000006
:1099C000AB9900000D800000576D00007A57000031
:1099D00097F50000BE3C0000A1570000E1500000D8
:1099E00030A10000CB0B000054270000A636000079
:1099F000192C0000463A0000A4AB000006520000FB
:109A0000030300007BDE0000D6F90000E1C1000086
:109A10000F8E000015D9000060500000034C0000BC
:109A20008B340000A0E20000031500003676000031
:109A300088330000151A000061A80000725400006D
:109A4000483A0000249A000058720000F1FB000020
:109A5000B1EC0000CE4F0000D0F50000660A000017
:109A60008CAE00008609000079AD0000E0690000BE
:109A70006E3A00001172000070160000885000005D
:109A8000DD6F00007FEB0000963400005E120000E6
:109A9000AC870000896800001F260000CD9C0000F4
:109AA0009A94000017A600009CFC00004BE5000003
:109AB000AB010000A2B10000C9F10000BBF400003E
:109AC00051CD00009C4B0000529D00008AAC00006C
:109AD0006A800000EAB4000074E8000083610000BE
:109AE00061D20000F7B70000863D00001564000059
:109AF000B3C20000219A0000A1E20000023E000073
:109B0000DC48000064B6000096D4000045D8000090
:109B10005FC800006FD20000FD79000062D2000033
:109B2000BF270000CAA900006A650000A6A80000BF
:109B30008B310000496200002031000066460000C1
:109B400051E6000001E8000071110000F2CA0000B7
:109B5000796A0000CBC1000058D10000C6CA0000DD
:109B6000542C000094E00000E904000069030000A8
:109B700063D0000011F40000C5640000A2D600000C
:109B8000874700003C1E0000DF45000064D900004C
:109B90008E6300004F55000013D4000076D3000000
:109BA0004C8C00001D4B000048FB0000D8DF00007B
:109BB000D08200003C7000007FFF0000001F00000A
:109BC000D35200001D34000054FD0000B2690000B3
:109BD000D4C50000F506000090D80000963C0000B7
:109BE000AC2D0000622C00007E5B00006043000092
:109BF00088B2000019320000BA8F0000D195000031
:109C00009522000079520000312D00002CE1000067
:109C10004AEA00001A75000032EF00007DAD000036
:109C2000B0F3000016EB000088100000E4F500001F
:109C3000F34500001CB00000D3480000F03C0000D9
:109C400061150000EFDD00002EC80000481F000075
:109C500053890000197100005D8F000084560000D8
:109C600056B800009A3F0000FDA30000524F0000CC
:109C70004CA600003A39000094B1000028580000BA
:109C8000907400009F30000037380000BCC900000D
:109C9000788F0000872B00008450000053D700000D
:109CA000431D0000522A0000A59C000098A400005B
:109CB0003B010000B1360000BEFD00002F8C00000B
:109CC0009E97000023AF0000A05600008ABA000053
:109CD0000EC90000E4B90000D218000031220000D3
:109CE000DB750000FDE0000030D400001C25000002
:109CF0009CCF000056D500000F4A0000E23600005D
:109D00002CE1000099490000E7B00000E98B000059
:109D1000473A00005D3B0000119F0000C66900004B
:109D2000D3D10000B6660000D41000004D1700002B
:109D30006B3200005356000043180000BBAD00001A
:109D4000544900002DC70000886B000003F7000095
:109D5000E0AE000083DE000069720000E57A0000DA
:109D60000A4400009A2700008F5C00004AB20000FD
:109D7000B2D800005BBA0000BA5C0000D940000015
:109D8000F00D00006C600000994D00002E7D000079
:109D9000413300009A5A000099FD0000D1010000F3
:109DA00052B10000B965000006FB000002BE0000D1
:109DB0009E580000D57800001B890000E2A2000038
:109DC000CAA00000A4CE0000AA420000E98C000056
:109DD00014A8000073B800000DBF000066DE00008C
:109DE00062F60000BF960000191F00002B1B000048
:109DF000692E0000C5AF00001B2C000055B5000007
:109E000068070000C8380000733F00008FDA0000C8
:109E10002AE60000DC51000097CF00001AC90000BC
:109E20002CB300003CA30000F58B0000C8E8000044
:109E30000349000036E90000F2180000D1AB000031
:109E40006BE30000AB8B000024A1000082580000EF
:109E50009EA80000AEB700005760000034B20000BA
:109E6000A85B000030E70000F6C90000FF0000001A
:109E70004E0B000028EB0000296A0000E30D0000F3
:109E80004D5100000CA800007F72000040C000008F
:109E9000FDF800007E480000E3920000C5A300002A
:109EA0004723000095C50000F1A20000315D0000CD
:109EB000A29200006DE9000091720000DA28000013
:109EC000F2FA00004118000063730000DE92000007
:109ED00046F8000099BA0000B1FE0000B61B000071
:109EE00062A700002FAD0000399E00007F24000013
:109EF000B7B500002534000024C500007E440000F2
:109F000096B100007FA0000036F20000C7B3000049
:109F1000FAE300003CCD000097D300009BA80000AE
:109F2000B1A8000071D400007EEF0000A93C000041
:109F3000FCB100000B2E00005BFB0000CC310000E8
:109F40008DE70000923A000071FE000040B700006B
:109F500063FC0000248C00005D09000052FB00003F
:109F6000522F0000F2B00000D3B40000B5AE0000E4
:109F70000EAA000086EE000083F60000500B0000E1
:109F800028F90000DB570000FA8E00003E6A00004E
:109F9000F6D3000056D2000071FE000066550000A6
:109FA0008EA40000ECE300005B7F0000947F0000C3
:109FB000D71F000052850000D3DD00005D80000047
:109FC000D87C0000B1F200007F160000535400005E
:109FD000710700001F66000070500000C665000099
:109FE000A8A80000AC65000045F40000240B0000A8
:109FF0009F4100008CBE00005C9200008ECD0000EE
:10A0000058560000EC1F0000A58600004A8A000098
:10A01000768E00000D4C0000F21500008D3400001B
:10A02000A9620000C7500000E4060000E71A000023
:10A030009FB300004F660000EEB5000090D700000F
:10A04000E7310000AB32000010C90000111D000014
:10A05000D8F70000BF7B0000A13E0000436C000069
:10A060001CFB00003DF600007F4B0000C3300000E9
:10A070002D450000605A00009CD10000ACC50000D6
:10A08000CF280000B6E40000BE1D000077EB000002
:10A09000E0300000706C0000809600002A00000094
:10A0A000DC92000040FA0000DFF10000C79E0000D3
:10A0B000CFE70000BFFC0000F197000094B600005D
:10A0C00045CC0000DCC50000461A000023A40000B7
:10A0D000EB8C00006C2E000000D6000007CB0000C7
:10A0E0006BE20000448A00005A160000546300002E
:10A0F000AAD80000C9B80000C3DA00001356000057
:10A1000067940000993E00004A4F0000BB0A00001F
:10A11000A8A300009E7200003F69000069060000CD
:10A12000CA0E0000E07A0000EF8D000071370000D9
:10A1300051BF0000317300008C390000714B0000EA
:10A140001A4E00007ECA0000C96D000010720000A7
:10A15000DA360000A7D40000CE41000076EB000004
:10A160007C4F0000C7AE00000EC00000827C0000E3
:10A170002F860000CCA80000265800008B77000036
:10A18000D85D000057CB000008EC0000A8E60000F6
:10A19000283800009CC100009B700000C6730000BE
:10A1A0004D1300006A260000091400008B1D0000FA
:10A1B0008D890000C5C5000078940000D2CA000057
:10A1C000B0DB0000B420000081E300008A7A0000C8
:10A1D000089A0000189A000099E20000EFCC0000F5
:10A1E000AC5C000013F0000044050000872F000065
:10A1F00013870000E28A0000752F000068B4000099
:10A200004F9700009D88000047620000790F000012
:10A21000CFFE00009889000016C8000001F0000081
:10A22000BE1500002BB000008E4B0000FDA6000004
:10A230000AA30000E7BF0000DD8E0000DBA70000DE
:10A24000963D000002DA000046950000D1EC0000C7
:10A2500070830000B6DD000031D10000CF1C00008B
:10A260002A4F00002C18000091BA0000433D000066
:10A270009EDC0000861C000054D8000061D0000065
:10A28000BB630000A2DC0000B1AC0000C5670000A9
:10A2900011450000B7C700004A0C00002AC40000A6
:10A2A00073C70000B97A0000620000006D940000DE
:10A2B0000187000028AA000024A30000AB8A000048
:10A2C00078180000ACA80000F70D00008E730000A5
:10A2D0003E580000E69D0000EF8800000356000095
:10A2E000CC1A00002E230000E1B40000CDA900002C
:10A2F000557D0000F2040000B48800007AD8000008
:10A3000077870000D7970000961E0000CA3D000026
:10A31000982E000071EC0000A0F10000ABE70000F7
:10A32000D57100004C290000A79C000052AC000031
:10A330002B6F0000D5BB00002DAF00007BFD00009F
:10A34000918000008E0D0000CE9B00002C9E00002E
:10A350006A69000098FB0000B54A00001461000023
:10A36000D0350000B6380000FA070000838F0000E7
:10A37000FF0000000B0F0000A0FF000000F4000031
:10A38000FAC200003FFD0000B2E100006D53000082
:10A39000261800006DA6000000FB000054F6000027
:10A3A000747800003B2B0000CA780000927C00000B
:10A3B000F6A3000032950000AA210000A5EC0000E1
:10A3C000E5850000542A000095660000BDC100002C
:10A3D000BFD90000B6020000F8430000296E00005B
:10A3E00025E300002CA3000021350000925000005E
:10A3F0008AD20000EC66000089060000B5D000009B
:10A40000AF6D000089FF000000080000C6FD0000DD
:10A41000FDA00000726A0000BCFF00000081000087
:10A42000B873000029CB000004260000AEA700008E
:10A4300034A600008E2100002B5900003576000064
:10A44000521D0000CDBC000006000000B813000043
:10A45000D9D7000013F0000097B40000CE1400001C
:10A46000CCB8000080E50000E2990000E79600000B
:10A47000994D00002CED0000236A000030CA000056
:10A48000C0900000540000002CA40000616E000089
:10A4900036CD0000D097000005F5000027710000C0
:10A4A00087B20000ACCB00002A97000022A5000074
:10A4B0008B8900006B2B0000D3340000CC630000BC
:10A4C000A29A00004961000050D10000210C000058
:10A4D000FA8500008EF60000296C00002BDA0000DF
:10A4E0002704000067DC000015C30000716600004F
:10A4F000196F000016E60000798D00004BD50000B2
:10A50000434700000D340000B18500005264000094
:10A5100060820000FBF80000918D0000DDE3000088
:10A5200083350000CC740000CA3B0000D95D0000F8
:10A5300062BA0000FA98000076FF0000009A00005E
:10A540007E98000009F60000AD580000B9870000B1
:10A5500007700000A55A00000EED00004E790000C3
:10A5600095CA0000BFEA00009D0F0000E0700000E7
:10A5700054220000BA0300009CA50000FA760000F7
:10A580000B430000EC720000811E00008A0C0000EA
:10A59000F78B0000B3840000CF6B000083940000B1
:10A5A000481E0000248E000046510000760A00007C
:10A5B000A509000020030000BEE3000001540000D4
:10A5C0005ECD0000B3EC0000EBDA00001663000083
:10A5D000C2190000B66F000023650000D97C00009E
:10A5E0004B5500002D620000A8D700002C4F000042
:10A5F000F0050000537B000031200000DFA00000C8
:10A60000B1220000FCB10000B9710000601F000021
:10A61000F69F0000C0BD000036AE00001B7F0000AA
:10A62000F8460000119500002FFE0000FAB8000067
:10A630008EDD0000724A00001FF90000B51800000E
:10A640001C230000FC2E0000B34D00002AB30000C4
:10A65000361E0000C8720000BC97000027CD000025
:10A66000EB780000173B0000ACAB0000ACA0000092
:10A6700067590000E9EB00008473000046D2000037
:10A6800044B7000031F70000557400009B11000032
:10A690006F5D0000F157000047C20000D5D20000F6
:10A6A000FB3000007E3A00008B880000EBE90000E0
:10A6B0009FDC0000E4AB0000F7080000C058000079
:10A6C000C11700001A390000F2B80000C1DE000016
:10A6D0005FC30000BC420000D3F1000055470000FA
:10A6E0000E71000095150000251D00004E69000048
:10A6F0005325000045210000CAD60000A1E2000059
:10A7000096C0000015670000320B00005D55000088
:10A710000DAD0000D7CF000015D40000208F000041
:10A72000ECA70000293B00009FD00000D35C000094
:10A73000D80F0000DEF00000BFD300000E53000071
:10A740006B4200001C130000D95900009238000031
:10A75000972A0000A59500006FDF00008C390000EB
:10A76000B73200004F5B0000E2FB000085E900000B
:10A77000488D0000EADC0000DCBB0000384500002A
:10A78000FDD10000AF4E0000DF2400005B79000027
:10A790000C060000E4130000D63E0000474600000F
:10A7A000B1C300000A0E0000C94000002D260000C1
:10A7B000AE9C0000F4DB00006C5E000052D700008D
:10A7C000E6340000F470000053A40000F0460000DE
:10A7D00091A8000041A200002BDF0000BB6E00002A
:10A7E000A4F800007DF80000D0B30000423D000056
:10A7F000B32600002F1A000076D8000055990000FB
:10A8000057C1000097530000996600007163000073
:10A81000B22A0000EE5C0000F80F00001C6500008A
:10A820007C290000C33F0000A1AA000067CC000003
:10A830005E790000066B00003B3400008D240000B0
:10A840006D7E0000CC310000BD8700008F9F0000AE
:10A850008F9700002C1200003F6B00002D4B000072
:10A8600054550000D4C9000051310000160D0000FD
:10A870002150000010780000050000006D810000EC
:10A880006E340000E30A00006C8200002304000024
:10A890001A660000CC1B0000944400009B270000B7
:10A8A0009BDB000071E400003AE30000267C00001E
:10A8B0008B320000E28D0000F8F10000F05B000038
:10A8C000348C0000973300005AB4000064A80000E4
:10A8D000291D000044560000ED160000FB69000031
:10A8E000B5C1000007A80000D8FD0000318F0000AE
:10A8F000FB500000F68F0000EFF50000272200005B
:10A90000C8660000229800000B540000D42100000B
:10A91000BF690000E28A00007A800000799E000092
:10A92000B8040000CE380000C73C000031D500005C
:10A93000D07B0000D951000028FD00006C8A000087
:10A9400000760000D43700004D420000D65D0000C4
:10A9500080B700002DAC00003C3000003D950000A9
:10A960008D5200006BEA0000546F00007DCD0000A6
:10A97000F7F90000639F00008FC100008C270000E2
:10A98000CDF4000051450000390500007C1B00009B
:10A9900007BD0000716E0000530000001CEA0000BB
:10A9A00093D40000852100008FE100008FA60000F5
:10A9B000730A00008EC200009B500000205C000063
:10A9C00073F00000DED80000C23D00008CD0000013
:10A9D0007BEF00001A470000311D0000CA5800003C
:10A9E0005A5200004F890000EE0F0000C4E300003F
:10A9F0006FCE00005E3300004B220000C8E1000073
:10AA000074800000C49F0000B43C000006310000C8
:10AA100079ED00004B2200008A2B000091EE00002F
:10AA20008A7900002BDE0000093B0000DAA5000057
:10AA3000D4FA000022D10000CDDB0000A8C5000040
:10AA4000FD0500003BA60000A9EA0000ECD50000CF
:10AA500052010000A88E00004A3A000001E5000003
:10AA6000F9FA0000ED03000023CA0000CC520000F8
:10AA70001ACA000095220000422D00001C4D000063
:10AA8000FF00000074BE00001FE60000F3F90000A4
:10AA90000D860000F7660000E2F600002D7F000042
:10AAA000118C000053690000690B00001BA9000015
:10AAB00099290000E27900002523000042EE000001
:10AAC0007C4F000096200000C48F00001515000088
:10AAD0004D5D0000483D0000BC8A0000646000003D
:10AAE000DF640000693600005F900000FCF00000A9
:10AAF000A5220000BEB0000030B70000BA40000040
:10AB0000DDDB000072760000E83D000017F1000078
:10AB1000F96100009E2C0000A8F700004E1900000B
:10AB2000CD27000026DA0000699D0000BE7A0000F3
:10AB30004DB0000071E90000A8FF000000430000D4
:10AB40001ECF000093AA000088ED0000510700000E
:10AB50004BB70000DF6F0000E78E0000638E00003F
:10AB6000754E0000D6E40000A0030000F3070000CB
:10AB70001DC70000A25A0000A46A000047B10000EF
:10AB80002A9600009CCB000019610000C81B000041
:10AB9000622E00002DB20000EB2D00002A92000072
:10ABA000077A0000E79F0000CBF20000C188000098
:10ABB00025FC00002105000000630000853A00002C
:10ABC000DB170000BC1D00004F0500005677000099
:10ABD0001C5500005124000091980000D8940000FA
:10ABE0006E440000E2E60000BB2D0000A734000028
:10ABF00014F20000CF4300004B1500004FBD0000D1
:10AC0000221F0000773A0000D4A50000C5F500001F
:10AC10006F610000D7CF00001AD900008E800000BD
:10AC200080A40000EDB60000E71C00002BD400005B
:10AC3000EDBD0000B073000099F00000ED0C0000C5
:10AC4000F98B00004D4D000034700000D24400002C
:10AC50006D56000084EE000096170000DBD7000060
:10AC600012FF000000450000D00C0000CA51000097
:10AC7000051C00002E820000896400008C49000041
:10AC8000B02D000073B900003E1C0000B1090000A7
:10AC9000467700006DED00008EA80000B1DF0000D7
:10ACA000064F000015380000CD29000061A9000002
:10ACB000CBA80000635D0000324800007DDE00008C
:10ACC0004D440000D90900003F7E00002BE0000049
:10ACD000CAE9000022A900004AC700007D790000EF
:10ACE00069600000624B0000F7DD000089F8000099
:10ACF00008E600002DD400009E6300001014000040
:10AD00000FBA0000EA430000C80B000073380000CF
:10AD1000FA130000D8F7000015700000E66D00007F
:10AD2000EC8600004E0A0000CE73000068B20000FE
:10AD3000ACC10000229E00009A4E0000DDC200005F
:10AD40001657000066600000E9AB000063F10000E8
:10AD50007DC70000193B0000D2C700001475000039
:10AD6000469A00009E840000B2D600003A7F0000A0
:10AD70007820000000A20000D60000009231000000
:10AD8000072F00009E080000B3D80000BDFA0000A5
:10AD90009A970000B25B0000248B00000D8A00002F
:10ADA000D8F500001B9D0000F01A0000B0A90000BB
:10ADB000703600006F6F0000FC5D000096E7000039
:10ADC000393E00005F930000F0CE0000662A0000CC
:10ADD0002AE80000EA120000B27A0000AA19000076
:10ADE000AC2900009155000090590000D760000088
:10ADF0004EA30000B03D000030050000ECEF000065
:10AE000034A80000CAFD0000A5F00000FD4F0000BE
:10AE100012710000056B000050400000F2B4000009
:10AE200087310000AB7700008E260000ECDC0000CC
:10AE30002FC60000DB1E0000F1F40000BDB90000C9
:10AE4000E08F000031CB0000E9280000286A0000F4
:10AE5000A7A300008A38000043C00000C9270000F3
:10AE600064050000BC540000DADD0000081B00008F
:10AE7000F86000004EAB00002AB4000008F30000A8
:10AE8000D2330000C77B00002D9000009403000027
:10AE9000C48B0000DAFE000043E600006F8C000067
:10AEA000D36D0000743F0000C5CF00000CB100005E
:10AEB0006A5A000036FA00001F6900007C2F00006B
:10AEC0000F160000F16B00002F100000E586000057
:10AED000964A00005A69000069640000EDD4000041
:10AEE000ACAE000011D50000829B0000EE7B00009C
:10AEF000AB800000EE2B0000E38C00009E5F0000A2
:10AF0000629C000020940000199D0000156E000056
:10AF100075420000D95D00004CB40000314C0000C7
:10AF2000AD360000A8F4000033290000506F000087
:10AF3000704500008E3300003A58000072E80000AF
:10AF400024860000695000004B160000B2CE0000BD
:10AF50004C460000C82D0000A7710000CB9F0000E8
:10AF6000A1F50000C4F9000072EA000025280000E5
:10AF7000292A000029CC00008EEA000091950000EB
:10AF8000BEAD0000D87D0000AF1F00003DB700003F
:10AF9000C29F000092D30000AA3600002F1E0000BE
:10AFA000357C000091F4000008E20000DE0C000097
:10AFB000E20A0000FC8F0000890700001350000027
:10AFC000D31C0000AC4C00007DDE00005995000051
:10AFD0001BF5000089A40000AB82000041160000B0
:10AFE000B1C0000076430000ED370000275F00008D
:10AFF0006C190000BE670000592F0000B9E4000082
:10B0000095F4000090D0000052D700004EA600003A
:10B010003477000088B300005C930000C81E000075
:10B02000D18000003E420000FBE300002CF600004F
:10B030009DC3000051650000AB4700009CC20000AA
:10B040000CD5000008E2000009A1000061AB00007F
:10B0500058010000983000003E40000079E20000F6
:10B06000A0560000E5320000D1C5000025470000D1
:10B070006D2800007EEA0000DC8B000036FC00003A
:10B080008DED0000D79F00009E1A0000F26A0000BC
:10B09000E2AC000056380000464E00009BA40000C1
:10B0A0007D290000957100004704000070DD00005C
:10B0B0004F10000052AF000015E50000924F000055
:10B0C00099D40000CB99000030330000A054000058
:10B0D000322A0000AE9D000040D80000FC3F000076
:10B0E0008F96000001E80000F8C3000086CF000042
:10B0F000F66E0000932300005CF700002EFD0000B8
:10B100002CD9000054B00000AD2900009D4C000077
:10B110009ACE0000A21700004DF7000026F80000AC
:10B12000C7AB0000326A00005121000099400000C6
:10B1300030CB000067520000B6220000DD050000A1
:10B14000FD6F00008B7E00001AE10000FA6A00002B
:10B15000B9E500006AA80000A5110000E85B000046
:10B160006C030000482F00007D7A0000C8E5000055
:10B17000CF71000083CD0000FF0000000A380000FE
:10B18000A52A00004EC200005E090000CD24000088
:10B190005A7C0000A72700008E8E0000A26A0000E3
:10B1A0009A880000B5A100008C0D000031810000DC
:10B1B000F106000027960000F73F000031830000F1
:10B1C000E1930000E68C0000374A000058AF000011
:10B1D000FBF20000927E0000817100005593000098
:10B1E000E52700002F9000004F9400003BC40000B2
:10B1F000CA1800006EDA000093BD000062760000FD
:10B2000037BE0000EBD20000DC8600002FE9000012
:10B21000733C0000D21600001EF300004EB3000085
:10B220000BFC000050320000A83E0000A0DB000034
:10B23000F1C30000B128000055CC0000ACDC0000D8
:10B24000D740000067B40000DABA0000FE16000024
:10B25000C912000054AA0000A65A0000AA890000E2
:10B260003B180000D523000062400000E6480000C3
:10B27000DC72000036E900008C200000BBCD00002D
:10B280003F6900003333000048E60000EEE40000B0
:10B29000DEE60000FE3D000071B30000FB4F000041
:10B2A000C8380000838B000073A800001E8E0000C9
:10B2B0009A380000F2FA000068F4000044B200007E
:10B2C000CC0300001277000063B100003B5E000079
:10B2D000C3E50000816A00003F650000B9E000009E
:10B2E000951E000069680000A3000000DEDA00007F
:10B2F000C9B70000DD8500004F8F00002FA90000B6
:10B3000065CA0000BEC600006958000075E600006E
:10B3100015640000F20F00006FA60000D891000035
:10B3200096C600001A9B0000591F000011D50000AE
:10B330008D1A00003F63000095800000BBD500001F
:10B34000669100008D440000B1090000116B0000FF
:10B350001EBC0000CFAE00002C6900007D980000EC
:10B3600052C5000012A30000663500000C07000063
:10B37000EEA000001F88000038320000648C00003E
:10B3800059790000EC62000008F20000CC8E000049
:10B39000B3350000AF3D000099AA000092CA00003A
:10B3A00048DC000022F4000003AF0000789C00009D
:10B3B00013D60000555400006615000049380000FF
:10B3C00091E90000E38900008B420000AA400000E0
:10B3D000B79B0000743F00008621000050E500008C
:10B3E000CB4F0000052D000032C80000CF0C00003C
:10B3F000004500000A390000002D000085AF000064
:10B40000B0170000D8730000E989000055A70000BC
:10B41000DD59000063EF00003CAD0000FB3500008B
:10B42000B6EC00007D310000856000008A930000CA
:10B43000C9320000CA140000EE450000AE5B0000F7
:10B440009D91000034540000D5FA000016690000F8
:10B450000E980000A45F000085CD0000AE41000002
:10B460001CC10000389D000054EF0000572B000065
:10B47000D2D20000BB220000ADBB000069BA0000C0
:10B48000ADFE0000CAF8000093D70000A7CF00006F
:10B4900014D400009944000072A300004935000054
:10B4A00064A9000051220000E921000000220000F0
:10B4B000317B000080B7000016B80000E7AB000049
:10B4C0006BF900006C010000252C000011D3000076
:10B4D00040910000442C00008A360000B5CD0000E9
:10B4E000CF8E0000FBFD000077FA0000EDC90000E0
:10B4F000CEE10000CEE00000669300004DE80000C1
:10B5000054310000A4480000A91200002A200000C5
:10B51000160A00003A0F00000FCF0000017E000065
:10B52000D86B0000FDCF000081EA0000541B000032
:10B530003D4C00008B000000F99B0000FE00000065
:10B54000E0DF000018B70000B7FC0000C6F50000FF
:10B55000541900007AB7000076280000DE6700006A
:10B5600003C40000ECBF000081FA0000E0F8000016
:10B5700091E700009430000056CC0000763E0000B9
:10B58000F1660000BF3600003FD70000E1850000F3
:10B59000E13100008B200000039D000081C200000B
:10B5A000B1DD0000669300008DF000009C580000A3
:10B5B000CD290000A71100004776000016410000C9
:10B5C000D7CC0000E2B400005FB600000C4D0000D4
:10B5D000C12100006D8E0000E71A00005EBD000072
:10B5E000C3290000EE800000B86600003565000049
:10B5F00064E80000D1F800002E9E00008F2F0000AC
:10B600004873000039B40000C9230000C4400000A2
:10B610008CB800000B6200006C390000DFA5000050
:10B62000B04F000010CB000028690000CC50000093
:10B6300051520000C51C0000CCBA000098CA00009E
:10B640000EBB0000346400009F2F0000888F0000B4
:10B65000962A00004C31000068FD00009A7C000032
:10B6600023EC00008F0C000036CA0000A4A00000EC
:10B670002A080000DF6B000079E300004519000094
:10B6800051410000C5340000CBEF0000734E0000B4
:10B69000273100001AA2000018A700006A34000039
:10B6A000B28300006DD7000099B50000AF8B000099
:10B6B00008B300004A2E0000DDDA000064850000B7
:10B6C000A26800005699000090D40000A1BA0000C2
:10B6D00029DA0000E4730000B8270000972B00006F
:10B6E000621F000010460000852900006E8A0000DD
:10B6F0007E5E000078AB000058620000BFEC0000E6
:10B7000093F800004622000003640000BCC3000060
:10B7100030CB0000A068000026CB000068E10000EC
:10B72000864E0000F2B60000997500001EF400007D
:10B7300043CB0000FC470000F84E000007A30000C8
:10B7400090A100008C8B000090A4000032A90000A2
:10B750003B5F0000169D00008C5700001FAB0000EF
:10B760004E5F0000BA3C0000309600008A3B0000AB
:10B770007ECD00003F84000060950000B3B2000061
:10B7800066D000004E9300002D550000219500006A
:10B790001E7600009D740000CA5700004DC70000CF
:10B7A000A6200000CB34000006600000D4D00000CA
:10B7B000182300001B68000032160000DC6F000038
:10B7C0007E580000926300004FDC00005FA600007E
:10B7D0003BD90000A5BE000005FA00006201000090
:10B7E0009AC700000B55000026690000C3B1000095
:10B7F000ACC100005D9500004C3200000F1000004D
:10B8000005B100009FF1000097110000E7900000D3
:10B81000F12500005463000031A800005EC800005C
:10B820002C6000001B0500000A14000001A40000A9
:10B83000741D00007E78000032F6000068070000EA
:10B84000B8D600000B0B00006A5F0000CF020000BA
:10B85000FED30000234F0000F8AA00005EE20000C3
:10B86000FEC500003A7A0000E2B10000FD190000B8
:10B87000B1FE0000E8B50000E06C0000E6A70000A3
:10B880003DA60000AC4E000021AF0000AE9E0000BF
:10B890001899000042A4000044920000C4860000F1
:10B8A000E6390000731E000003120000A38D0000A3
:10B8B000BF490000D05A000029420000FBC200002E
:10B8C000B1EE00009D9400001DEF00006FBF00006E
:10B8D000027900002B340000593D00007B44000039
:10B8E0004A1E0000D62D0000D4DB0000A36100003A
:10B8F00094AC0000A9ED000047F7000089BF0000EC
:10B900008CE1000059B10000A9310000EB230000D8
:10B910008BD10000A5F10000CC250000E2A20000C0
:10B920008E8D000065A9000044690000890B0000AD
:10B93000CC5D000086C20000FE77000018C9000040
:10B94000331E000018AE0000A5CF00009A4500008D
:10B95000A3990000696300008FB700002106000072
:10B96000B48D00009B980000BADC00000F1D0000A1
:10B97000FCB00000FD4D000055410000700C0000BF
:10B98000F29000004AEC00005CF8000062E7000062
:10B990002076000034B5000020B1000020860000B1
:10B9A000077F00002C5B00001E3E00000B430000E0
:10B9B000633700002ECA00009A0C0000DE4C000025
:10B9C000A25F00007A8E0000133E00008371000029
:10B9D000114D00005DE30000C8810000F9E00000A7
:10B9E00093800000335C0000C33E0000CD73000074
:10B9F00019B3000084310000C4CA0000B22B00005B
:10BA0000B82400000D2400008215000047C4000087
:10BA10006E76000007960000F8A90000A08D0000D7
:10BA20000CD10000DD17000098E90000E78200005B
:10BA30002CAE000018D600000A020000B1A00000E1
:10BA40003B72000051E50000833D000021B800007A
:10BA5000D7DA0000CD0E0000873D0000CBE40000E7
:10BA6000630800002D090000416000005C2D00000B
:10BA70009ADD00007CBE000078760000B33F000035
:10BA8000CAE80000E3D500003D740000163D000048
:10BA900011B500001FA00000C0DC0000C8BE0000FF
:10BAA000F1510000DD1C00009BA70000AE03000068
:10BAB000EA5100003B370000EEAF000023D3000046
:10BAC000098B0000B34500009A23000071AE00000E
:10BAD00048BC0000A6910000BD2100006FE50000F9
:10BAE00086BF0000E38C0000A4230000155A00006C
:10BAF00096550000009B000045FC0000CE3300007E
:10BB0000C85100003B350000EEAF0000D30E00002E
:10BB1000944F000072A90000EEAF000021D3000096
:10BB2000FC58000031FD000001BD000006C7000008
:10BB3000DA16000052B60000D315000059B9000013
:10BB4000EA830000FF000000362C000044D3000010
:10BB5000D4D20000C75700004B420000EA92000018
:10BB60002EA0000092380000520700008EC700008F
:10BB7000197D000024710000FBE500003F7100000A
:10BB80007F6A00009D3C0000F1BC00002AAF00006D
:10BB900065F000008E430000A7A600000BD0000057
:10BBA0002327000060EE000054B50000753200004D
:10BBB000F69E0000EF120000A26D0000BCC700005E
:10BBC0009FF00000E2550000553B000053D50000F7
:10BBD00046ED0000A649000089010000E4F20000E3
:10BBE0003B5900007C39000062D300002155000061
:10BBF000EC6A0000B61F0000B63D00003C86000065
:10BC0000255600002AF600004FDD00001F0F00003F
:10BC10008639000059B20000CB6800004CA6000035
:10BC2000F68A0000916E0000BF7E00002D680000C3
:10BC300025D700000D980000F78700003C41000068
:10BC400020580000ED89000019780000FD790000FF
:10BC5000F4C70000364800005A2700009361000036
:10BC60007F0F00001C7C0000BFED00003B33000094
:10BC7000199F00001666000092A300000318000040
:10BC800093B000004B9E000088740000FE37000057
:10BC9000C7D4000052010000D9B60000DD31000019
:10BCA000F27500006A2300004A2E0000AA6F00000F
:10BCB000275100008DFF000000E3000062B9000082
:10BCC000363B00001F65000030E50000E98F0000F2
:10BCD0006FD300009E2E00007B0800006C7F0000E8
:10BCE000551F0000F08C0000244300001FFF0000DF
:10BCF000006D00003F84000063A8000038AE000023
:10BD0000A38C00004B5D00000AF400000DA80000A9
:10BD1000FA0C0000796A0000E32D000023480000BF
:10BD20007BCC0000E5B9000079E20000FB2C0000AC
:10BD3000862F00007BFD0000927C00000DF60000C5
:10BD4000462B000025A7000086EB0000FA980000B3
:10BD5000F97E0000E8C30000F169000008970000C8
:10BD600067FF0000D9000000000000000000000094
:10BD700000000000000000000000000000000000C3
:10BD800000000000000000000000000000000000B3
:10BD900000000000000000000000000000000000A3
:10BDA0000000000000000000000000000000000093
:10C000000200FA009EC0A9000080EB0070248800A6
:10C010000080EB0050248800AA24EF0022002000BA
:10C020008000EB00C04A2000F9DD0700200020005E
:10C0300030258800A824EF008644A900F0092000DC
:10C0400080248800F00920006024880082C4A800B1
:10C050008804A800000021004800DE00C0248800F9
:10C060000040EB00004F7800070037001E80FB0007
:10C07000C200DD0000002100008140006000B80027
:10C080000089BE001E4FE8001E407800E74F5000B8
:10C09000F6FF36009424A8009624EF0094A4A9008B
:10C0A0009424A9008000200050248800E0C52000CE
:10C0B0008040EB000148780040C620008040EB0043
:10C0C0000148780021638000F00F200000806000AC
:10C0D000206388003163800000F02F000080600042
:10C0E0003063880050248000680060000000E00099
:10C0F000ECFF3A0010C0B3003DE8B70010C0B30039
:10C100003EE8B7003F68EF004068EF003768EF0097
:10C110000040EB00004F7800170037001E80FB0046
:10C1200080004000E0822000008040008000EB00A2
:10C13000010878001E80FB0080004000A0822000E3
:10C14000008040008000EB00010878009E80FB002A
:10C15000A0C62000008040008040EB00014878002D
:10C160009E80FB00C0C62000008040008040EB00A5
:10C17000014878001E4FE8001E407800E14F500053
:10C18000E6FF36008000210070418800D0002000CA
:10C1900050258800E0C620001080880000002100A3
:10C1A00081C0B300014878001000210041C0B300F5
:10C1B000014878001000210010407800804078008D
:10C1C0000174A00010002100014878002468EF00ED
:10C1D0004228EF004428EF004668EF002228EF00D5
:10C1E0000080FA00000006000200FA001041800002
:10C1F0000000E00013003A009424EF008C24EF00CC
:10C200002000200030258800A824EF008644A900E3
:10C21000F009200080248800F009200060248800B4
:10C2200082C4A800010037009404A800A024800064
:10C23000610060000000E000FBFF32001000200001
:10C240001041880010418000E10F50000C003A00BE
:10C25000A124800000042000008060000000E000B5
:10C2600007003A000080EB00502488008C24EF0087
:10C270008C04A8008C84A8002000200010418800B5
:10C2800000248000700060000000E0000700320021
:10C2900010248000700060000000E0000300320005
:10C2A00000012000002488009E0407004024800034
:10C2B000620060000000E000020032008EC0A900B1
:10C2C000A200370050248000610060000000E00000
:10C2D0000900320060248000610060000000E0007E
:10C2E0000500320046FF0700400020001041880092
:10C2F000100020005024880050248000700060004E
:10C300000000E00005003200602480007000600042
:10C310000000E000010032007504070001248000E5
:10C3200000042000008060000000E00003003200F4
:10C330000004200000248800D50607005024800057
:10C34000640060000000E0001400320060248000FF
:10C35000640060000000E0000400320012002000D1
:10C360008000EB0030072000360F0700400020005F
:10C37000502488003BC8BF000004E00003003200E6
:10C380003BC8BF000040E9003BE8B7003BC8BF0026
:10C390000004E00001003A008501070051248000FC
:10C3A00000082000008060000000E000060032006D
:10C3B0006124800000082000008060000000E00090
:10C3C000010032002E04070050248000620060004B
:10C3D0000000E0000C003200602480006200600079
:10C3E0000000E00008003200120020008000EB0096
:10C3F000F0FF2700130F07000080EB007024880077
:10C40000200020005024880010418000E30F5000DD
:10C4100002003E008EC0A9004C003700602480005E
:10C42000680060000000E000470032000040EB00C0
:10C43000004F78003F003700502480006800600003
:10C440000000E0003F0032009024800000407800AF
:10C4500038E8B70038C8BF000080FB004400DE00A9
:10C460000040780039E8B7008000200050248800A0
:10C4700038C8BF00684060000004E00012003A00C5
:10C4800039C8BF000081FB0039C8BF008080FB00B5
:10C49000C0C62000008040009040780061C060006D
:10C4A0000004A200E1406000C0C62000000041007E
:10C4B000E1C06000104178000204A10081407100D9
:10C4C000014878001100370039C8BF000081FB0027
:10C4D00039C8BF008080FB00A0C62000008040005B
:10C4E0009040780061C060000004A200E14060005C
:10C4F000A0C6200000004100E1C0600010417800AB
:10C500000204A100814071000148780039C8BF00D1
:10C510000004E00002003A000E04070004003700A7
:10C520000001EB008183200020072000C50E0700DA
:10C530001E4FE8001E407800E34F5000BEFF36005B
:10C5400001003700000000008EC0A9000080FA0042
:10C55000000006000400FA002047980031479800C8
:10C560003E4090000080FB00680060000000E0009A
:10C57000030032008040EB002E4090007B0107005A
:10C580003E4090000080FB00640060000000E0007E
:10C590000300320011C0B3002E4090007301070069
:10C5A000A14A20002E4090000080FB0000004000C7
:10C5B000008F40001E007800BE40900001487800C7
:10C5C0000080FA00000006000800FA0020479800EA
:10C5D0003147980022079800634798003E4090003A
:10C5E0000004E000070032002E4090000080FB00B5
:10C5F00080004000E082200000804000100F7800A2
:10C60000060037002E4090000080FB0080004000B4
:10C61000A082200000804000100F78001E007800EB
:10C620000000E00002003A000000EB003700370095
:10C63000AE0090001E007800110098001E007800E7
:10C64000EE409000014878001E00780010409000F5
:10C6500002C4B300824060001E00780011409800C0
:10C660001E00780010409000804078000134A00047
:10C670001E007800114098001E00780010409000C5
:10C68000804078000174A0001E00780011409800DE
:10C690003E4090000004E0000E0032002E4090006A
:10C6A0000080FB00AE4090008180FB0001814000D3
:10C6B000E182200081004100910078000120A20069
:10C6C00000014000E08220000000410001087800E5
:10C6D0000D0037002E4090000080FB00AE4090001F
:10C6E0008180FB0001814000A18220008100410087
:10C6F000910078000120A20000014000A0822000EB
:10C7000000004100010878001E0078000080FA0057
:10C71000000006000400FA00204798003147980006
:10C720002E4090000004E00017003A0040418000D5
:10C7300081C0B3000148780040418000E1C620007C
:10C740001100980040418000C1C0B3001140980022
:10C750004041800041418000914090000174A00060
:10C76000114098007041800041C0B3001140980012
:10C770007041800071418000914090000174A000E0
:10C78000114098002E0037002E4090000080FB00E2
:10C7900000004000800078003E4090000080FB00D8
:10C7A000008040004300DD00800078000000210090
:10C7B000008F40001E0078001040900080407800FC
:10C7C0000124A0001E007800114098001E0078008F
:10C7D00010409000804078000174A0001E00780096
:10C7E000114098002E4090000080FB0000004000A7
:10C7F000800078003E4090000080FB0000804000F8
:10C800004300DD00E400400000002100008F4000F4
:10C810001E00780010409000804078000124A000A5
:10C820001E007800114098001E0078001040900013
:10C83000804078000174A0001E007800114098002C
:10C840000080FA00000006000200FA00004F7800A5
:10C85000A124800000022000008060000000E000B1
:10C86000510032001E80FB0080004000E08220006A
:10C8700000804000100278001E80FB008000400015
:10C88000E082200000804000100078001001BE000F
:10C8900000042000010020008202780003017800DB
:10C8A000800178000100780083826200000061004E
:10C8B0008000EB00C000DD00000020000001BE0091
:10C8C0006128B8000001710081817100028ABE00F8
:10C8D0001E80FB0080004000E082200000804000BD
:10C8E000100278001E80FB0080004000E0822000E3
:10C8F00000804000100078001001BE0000042000FD
:10C90000010020000000690081806900008ABE00EB
:10C910001E80FB009E80FB0001814000E182200020
:10C9200081004100910078000120A2000001400038
:10C93000E082200000004100010878001E80FB001A
:10C9400080004000E08220000080400090007800DD
:10C950001E80FB0000014000E0822000000041003A
:10C9600010007800104090000044B2009040980001
:10C970001E80FB0080004000E0822000008040001C
:10C98000900078001E80FB0000014000E082200043
:10C9900000004100100078001041900000C4B30076
:10C9A00000406900904098000080FA0000000600F6
:10C9B0000000FA003DC8BF000004A2000004E0002F
:10C9C0003400320010C0B3003DE8B7003EC8BF00DD
:10C9D0000004A2000004E0002E00320010C0B300EA
:10C9E0003EE8B70033C8BF00E24F50000C003A00E9
:10C9F000704180008040EB00014878007041800069
:10CA000081C4B300114098007041800071418000E2
:10CA1000914090000174A000114098001D00370063
:10CA200033C8BF00E14F50001A003A003A68EF00E7
:10CA30003041800081C0B30001487800304180005F
:10CA4000E1C62000110098003041800041C0B300D1
:10CA500011409800304180003141800091409000A9
:10CA60000174A0001140980010C0B3003AE8B7006C
:10CA70004041800081C0B3000148780040418000FF
:10CA8000E1C62000110098004041800001C8B300B9
:10CA9000114098000080FA00000006000000FA0033
:10CAA0003F68EF004068EF0033C8BF00E24F50001E
:10CAB0000F003A004041800081C0B3000148780077
:10CAC0004041800061C72000110098004041800073
:10CAD00081C4B30011409800404180004141800072
:10CAE000914090000174A000114098001D00370093
:10CAF00040C720001080FB0051C720009180FB0040
:10CB0000C808DD000100700080007800006380002C
:10CB1000808F50000700310040C720001080FB00CC
:10CB200051C720009180FB00C808DD0001007000A3
:10CB300000638800960007007041800061C72000F4
:10CB4000110098007041800081C4B300114098002A
:10CB50007041800071418000914090000174A000FC
:10CB6000114098000080FA00000006000400FA005E
:10CB7000204798003147980000002100000F7800FE
:10CB80002E4090000080FB000000400080007800F4
:10CB90003E4090000080FB00008040004300DD002C
:10CBA0001E0F40001E0078009000780001F0A100E8
:10CBB000010878003E4090000004E00007003A00C1
:10CBC0002E4090000080FB0080004000A0822000EA
:10CBD000008040001E087800060037002E409000BC
:10CBE0000080FB0080004000E082200000804000C8
:10CBF0001E0878001E0078009000780001E0A10077
:10CC0000010878009E007800648040009000780061
:10CC100001E0A000010878000080FA000000060092
:10CC20000000FA0094A4A900F1628000000820002E
:10CC3000008060000000E00027003A0040C62000AD
:10CC40009040780000C8B30000C060000004E0001D
:10CC50000A00320020C0B30033E8B70040C8BF006C
:10CC60000004A2000004E000010032008BFF070076
:10CC70003E68EF003D68EF00430037004041800010
:10CC800081C0B3000148780040418000E1C6200027
:10CC90001100980040418000C1C0B30011409800CD
:10CCA0004041800041418000914090000174A0000B
:10CCB000114098007041800041C0B30011409800BD
:10CCC0007041800071418000914090000174A0008B
:10CCD000114098002C003700E0C6200090407800FA
:10CCE00000C8B30000C060000004E0000F00320084
:10CCF00010C0B30033E8B7003FC8BF000004A20073
:10CD00000004E0000100320064FF07003E68EF000D
:10CD10003D68EF003CC8BF000004A2000004E00032
:10CD20001900320022FF07001700370020C0B300AF
:10CD300033E8B7004041800081C0B300014878006B
:10CD400040418000E1C62000110098004041800071
:10CD500041C0B30011409800404180004141800033
:10CD6000914090000174A000114098003E68EF00CF
:10CD70003D68EF003CC8BF000004A2000004E000D2
:10CD8000010032000AFF07000080FA0000000600E0
:10CD90000200FA0080C0B300004F780000638000FA
:10CDA000E70F50000D003E0000638000004F780048
:10CDB00032C8BF000004E00003003A0010C0B30016
:10CDC00032E8B7000500370032C8BF00E14F50001D
:10CDD00002003A0020C0B30032E8B70001638000CF
:10CDE0001E80FB00008050000063880070418000BE
:10CDF0001E48780060C72000A0418800F0628000D3
:10CE0000610060000000E00017003A0009003700F0
:10CE1000A1418000E06280001041780082487800E3
:10CE20008100E800A14188000000E800E06288007D
:10CE30001E4FE9001E4078000004E000F4FF3A00B5
:10CE40000C003700A1418000E062800010417800B2
:10CE5000824878008100E800A14188000000E800D5
:10CE6000E06288001E4FE9001E4078000004E000E8
:10CE7000F4FF3A000080FA00000006000200FA0009
:10CE800030418000104F78009E80FB0020638000BE
:10CE90004800DE0033638000F20F20000281610051
:10CEA0004811DD0002007000808F5000080036003D
:10CEB000206380004800DE0032638000F10F200014
:10CEC00081006100C808DD0001007000004F78009B
:10CED000206380004800DE0032638000F10F2000F4
:10CEE00081006100C808DD0001007000800078004A
:10CEF0001E80FB0000805000F10F200081006000C8
:10CF0000C808DD0023638000F20F20000281610069
:10CF10008280700021638800C800DE00F00F2000CE
:10CF2000008060003263800001F02F00810061000A
:10CF300001007000306388000040EB00104798004B
:10CF40000C003700106380009E4090000181FB00C0
:10CF500061C72000810041009140780001487800BD
:10CF60000000E800106388001E4090000040E800C8
:10CF7000104798001E4090009E4F5000F1FF39006E
:10CF8000206380004800DE0032638000F10F200043
:10CF900081006100C808DD00010070000000E000B1
:10CFA0001E0032004041800081C0B300014878007B
:10CFB0004041800061C7200011009800304180008E
:10CFC0009000780000002400008060000000E00075
:10CFD00009003A004041800081C4B300114098002C
:10CFE0004041800041418000914090000174A000C8
:10CFF00011409800300037004041800081C0B300EC
:10D0000011409800404180004141800091409000D3
:10D010000174A000114098002700370040418000B3
:10D0200081C0B3000148780040418000E1C6200083
:10D03000110098004041800041C0B30011409800A9
:10D040004041800041418000914090000174A00067
:10D0500011409800306380004800DE004263800089
:10D06000F10F200081006100C808DD0001007000A0
:10D070000000E00008003200306380004800DE005D
:10D0800042638000F10F200081006100C808DD00CC
:10D090000100700000000100206380000070A1000A
:10D0A000206388003CC8BF000004A2000004E00028
:10D0B000010032003EFE07000080FA00000006007A
:10D0C0000200FA00F06280000070A000F0628800A8
:10D0D000220020008000EB00C04A2000CCD90700CD
:10D0E000020220008000EB0000002100C8D90700E8
:10D0F0009424A8000040EB00004F78000B0037009C
:10D100009E80FB00A0C62000008040008040EB0015
:10D11000014878009E80FB00C0C6200000804000CF
:10D120008040EB00014878001E4FE8001E40780068
:10D13000E14F5000F2FF3600120020008000EB00AB
:10D1400050822000B2D907009424A9008000210059
:10D15000704188000000210030418800304180008B
:10D160004041880000C720001040780024E8B70044
:10D1700024C8BF000004E00003003A0000012000C2
:10D180001041880006003700120020004182200074
:10D1900010002000AB0B07000002200010418800A7
:10D1A0000080FA00000006000000FA00E0C620003F
:10D1B0009040780000C8B30080CF500047003A008C
:10D1C000E0C5200001CCB3000148780010C7200062
:10D1D000104078000080FB00E20F50000900320090
:10D1E000E30F500023003200E10F500037003A00F7
:10D1F00060C12900E06288002001200000638800EF
:10D200003600370000C72000104078000004E0001E
:10D2100014003A0000C72000104078000080FB0096
:10D22000000040008000780040CA290000804000D3
:10D2300010007800E0628800E06280000080E80072
:10D240009040780000C6200001487800E06280002D
:10D25000630040009040780010C62000014878002C
:10D260001E003700E0C520008040EB000148780038
:10D270001A00370000C7200010407800E34F50002C
:10D280000E003E0000C72000104078000080FB0028
:10D29000000040008000780060CA29000080400043
:10D2A00010007800E0628800E062800010407800A2
:10D2B0000080FB000063880008003700E0C5200004
:10D2C0008040EB000148780004003700E0C52000F2
:10D2D0008040EB0001487800000000000080FA0068
:10D2E000000006000200FA0060C720008040EB004A
:10D2F0000148780070C720008040EB0001487800AA
:10D30000E0C62000904078007FC060000080FB00F5
:10D31000E10F500011003200E20F50001300320004
:10D320000000E00047003A00F06280000070A000BA
:10D33000F062880036C8BF000004E0003A00320006
:10D3400060C7200010407800804078000114A000E1
:10D3500060C72000014878003A003700F062800082
:10D360000070A000F062880036003700F062800094
:10D370000070A000F062880020C7200010407800F4
:10D380006F4060000004E0002900320020C7200048
:10D390009040780000C8B30000C060000004E000C6
:10D3A00009003A0020C72000904078006FC060005C
:10D3B0000080FB0080004000A08220000080400030
:10D3C000100F78000800370020C720009040780038
:10D3D0006FC060000080FB0080004000E082200001
:10D3E00000804000100F78001E0078009000780048
:10D3F00000002800008060000000E0000E00320005
:10D400001E0078009000780000402000008060003E
:10D410000000E0000A00320060C7200011C0B30025
:10D4200001487800070037000000000005003700C1
:10D43000000000000300370000000000010037007A
:10D4400000000000F1628000000820000080600001
:10D450000000E0000800320060C72000E0628800A1
:10D46000F06280000000A000F062880000C620008A
:10D4700021C0B300014878000080FA0000000600D7
:10D480000000FA0050258000620060000000E0000B
:10D4900013003200304180009040900000C8B3007B
:10D4A00080CF50000D003A00704180009040900005
:10D4B00040C8B30080CF500008003A0030418000DF
:10D4C000C1C0B3001140980030418000314180005C
:10D4D000914090000174A00011409800AA24A90076
:10D4E00000082000502488000080FA000000060098
:10D4F0000000FA008284A800000120005024880067
:10D5000010C0B30037E8B7004668EF000001EB0039
:10D510008000EB0050072000CA0A07000080FA00D4
:10D52000000006000000FA003768EF000001EB0081
:10D530008000EB0040072000C20A07008284A90097
:10D5400000012000002488004668EF000080FA00F7
:10D55000000006000000FA00D0C2B3003BE8B700AC
:10D5600038C8BF000080FB000020A1000000E000E0
:10D570001F003A0038C8BF000080FB004200DE00F8
:10D58000004078000080FB00C200DD0000002100A8
:10D5900000804000304188003041800040418800D8
:10D5A000404180000020A2004041880030418000BE
:10D5B0009000780000C023008080600000402300BD
:10D5C000808F500008003A00304180001000900029
:10D5D0008200200080007800E0C6200085D8070087
:10D5E0000B000700080037003D0007000600370069
:10D5F00038C8BF000080FB000020A100E80F5000E9
:10D6000001003A00530007000080FA000000060005
:10D610000000FA003268EF003C68EF003F68EF005E
:10D620004068EF003A68EF003368EF007041800017
:10D6300071418000914090000174A1001140980058
:10D64000704180000020A20070418800704180007D
:10D6500071418000914090000174A1001140980038
:10D66000704180000020A20070418800404180008D
:10D6700041418000914090000174A1001140980048
:10D68000E0C520008040EB00014878000000EB007E
:10D690000063880040C620008040EB00014878000D
:10D6A00021638000F00F200000806000206388006C
:10D6B0003163800000F02F0000806000306388003C
:10D6C000830007000001EB008000EB003000200029
:10D6D0005C0A070052FD07000080FA000000060007
:10D6E0000000FA0033C8BF00E24F500002003A00C9
:10D6F000E2FD0700150037003368EF003AC8BF00AD
:10D700000004A2000004E0000F003200404180004D
:10D7100081C0B3000148780040418000E1C620008C
:10D720001100980040418000C1C0B3001140980032
:10D730004041800041418000914090000174A00070
:10D7400011409800010037003A68EF000080FA00AD
:10D75000000006000200FA0070418000100078000E
:10D760004E00DE0061406000004F78007041800094
:10D770000020A2007041880010418000E80F500096
:10D780000E003A0000C72000104078008080FB00A7
:10D79000F007200000806000B0248800B0248000E2
:10D7A0000000E0000300320000012000104188006A
:10D7B00002003700400020001041880033C8BF003D
:10D7C000E14F500025003A007041800061C7200001
:10D7D000110098006EFD070032C8BF00E24F5000F4
:10D7E00009003A007041800041C0B3001140980028
:10D7F0007041800071418000914090000174A00050
:10D8000011409800300037001E4078000004E0000E
:10D8100009003A007041800081C4B30011409800B3
:10D820007041800071418000914090000174A0001F
:10D8300011409800240037007041800081C0B3007F
:10D84000114098007041800071418000914090002B
:10D850000174A000114098001B00370040C6200052
:10D860009040780000C8B30000C060000004E000F1
:10D8700014003200306380004800DE004263800004
:10D88000F10F200081006100C808DD000100700078
:10D890000000E00008003200306380004800DE0035
:10D8A00042638000F10F200081006100C808DD00A4
:10D8B0000100700000000100206380000070A100E2
:10D8C000206388003368EF000080FA000000060043
:10D8D0000000FA00E0C62000104078000046B200C8
:10D8E0000004E00051003A00F0C62000104078002B
:10D8F0000080FB00CF80DE00B2002000030020008B
:10D90000820F5000838F58004A003E0000600100E3
:10D910002100370022003700480037002000370080
:10D9200046003700060037000B0037003A0037008A
:10D930000D0037000A0037001B0037002A003700AF
:10D94000F06280000070A000F0628800800020007B
:10D95000104188003A00370013FE070038003700F6
:10D96000D7FD07003600370040822000E0628800C3
:10D97000F06280000000A000F062880000C6200075
:10D9800011C0B30001487800F06280000070A00070
:10D99000F06288002A00370052FE07002800370096
:10D9A000290007002600370020C72000104078001B
:10D9B0008080FB005082200000804000E0628800F0
:10D9C000F06280000000A000F062880000C6200025
:10D9D00011C0B30001487800F06280000070A00020
:10D9E000F062880016003700F06280000070A0002E
:10D9F000F062880020C72000104078000081FB0002
:10DA000000C72000904078005082200000004100B4
:10DA1000014878000A0037000001EB008000EB00AD
:10DA200020002000870907000500370000000000E3
:10DA30000300370000000000010037000000000074
:10DA40000080FA00000006000600FA0000C720006F
:10DA500010407800E14F500010003A00E0C620006E
:10DA6000104078007F4060000004E0000B003A00A6
:10DA7000F06280000070A000F0628800F0C6200014
:10DA800010407800E34F500003003A0010C0B3008C
:10DA900036E8B700010037003668EF0000C7200005
:10DAA000104078000004E000F7003A00E0C62000D3
:10DAB000104078007F406000E24F5000F2003A00D2
:10DAC00020C72000104078006F4060000004E00094
:10DAD000ED00320020C72000904078006FC0600049
:10DAE0000080FB00E10F5000E7003C001141800086
:10DAF00000022000808F5000E3003A00F0628000B6
:10DB00000070A000F062880020C7200090407800DC
:10DB100000C8B30000C060000004E00011003A003B
:10DB200020C72000104178006F4061000080FB009A
:10DB300080004000A082200000804000100F78008C
:10DB400020C72000904078006FC060008080FB00FC
:10DB5000C0C6200000804000104078004047980078
:10DB60001000370020C72000104178006F4061008E
:10DB70000080FB0080004000E08220000080400028
:10DB8000100F780020C72000904078006FC0600020
:10DB90008080FB00A0C6200000804000104078007C
:10DBA000404798004E409000614060000004E00053
:10DBB00004003A001E0078000020A100000F780049
:10DBC000030037001E0078000020A000000F78003E
:10DBD00020C720009040780000C8B30000C060005B
:10DBE0000004E0000A003A0020C72000104178003D
:10DBF0006F4061000080FB009E0078000001400043
:10DC0000A0822000000041000108780009003700D0
:10DC100020C72000904078006FC060000080FB00AB
:10DC20009E00780000014000E082200000004100DA
:10DC300001087800F0C6200010407800E34F500043
:10DC40002C003A001E0078009000780000002800A8
:10DC5000008060000000E0001900320020C72000B2
:10DC60009040780000C8B30000C060000004E000ED
:10DC70000A003A0020C72000104178006F40610080
:10DC80008080FB00C0C620000080400090407800EB
:10DC90000114A000014878000900370020C72000C7
:10DCA000904078006FC060008080FB00A0C620001C
:10DCB00000804000904078000114A00001487800E6
:10DCC0001E00780010409000804078000124A000E1
:10DCD0001E007800114098001E007800104090004F
:10DCE000804078000174A0001E0078001140980068
:10DCF000650037001E0078000020A200000F7800A9
:10DD00001E0078009000780000002800008060006D
:10DD10000000E000110032001E007800104090006A
:10DD2000804078000174A1001E0078001140980026
:10DD30001E00780010409000804078000164A00030
:10DD40001E00780011409800220020009E007800FC
:10DD500050002000BB080700060037001E007800B6
:10DD600010409000804078000164A0001E00780000
:10DD7000114098001E0078000020A200000F7800DB
:10DD80004E409000624060000004E00006003A004F
:10DD90001E007800900078000000280000806000DD
:10DDA0000000E0002400320020C7200090407800EE
:10DDB00000C8B30000C060000004E0000A003A00A0
:10DDC00020C72000104178006F4061008080FB0078
:10DDD000C0C6200000804000904078000114A100DF
:10DDE000014878000900370020C7200090407800E3
:10DDF0006FC060008080FB00A0C620000080400053
:10DE0000904078000114A100014878001E007800BD
:10DE100010409000B2C3B300824060001E00780042
:10DE200011409800220020009E0078005000200041
:10DE300084080700060037001E007800104090009C
:10DE4000B2C3B300824060001E0078001140980009
:10DE5000A14A200020C72000104178006F406100D7
:10DE60000080FB0000004000008040001007980088
:10DE70001E00900010407800804078000114A1003E
:10DE80001E009000014878000080FA0000000600A3
:10DE90000000FA0010428000214280006100400032
:10DEA000E0804800104288002142880037C8BF0047
:10DEB0000004A2000004E0000800320046C8BF00D1
:10DEC0000040E80046E8B70046C8BF000004E00094
:10DED00002003A0000C0EB0046E8B7000080FA00FC
:10DEE000000006000000FA0010428000214280007D
:10DEF0000080FA00000006000000FA00E0C72000E1
:10DF000003C4B300000178008040EB0010C0B300F0
:10DF1000ADF90700404088008041800050408800F3
:10DF20000068EF0000C0EB0001E8B7000268EF00F6
:10DF30000368EF001168EF001A28EF001C28EF00BB
:10DF40001E28EF002028EF0010C0B30012E8B70031
:10DF50000E28EF0090EB20008040EB000148780095
:10DF60001F00370090EB2000104078008080FB00FD
:10DF700000812000008040008040EB0001487800D4
:10DF80002177800060778000010001000004E0003C
:10DF90000D003200F1768000607780000100010002
:10DFA0000000E0000800320090EB200010407800F4
:10DFB0000080FB00110020008008DD007040800020
:10DFC0000100700070408800C304070090EB20003F
:10DFD000104078008040E80090EB20000148780075
:10DFE00090EB2000104078000004E000DDFF3200DC
:10DFF0000080FA00000006000000FA00E0C62000E1
:10E00000104078007F406000E14F500054003A001B
:10E0100020C72000104078000004E00052003A00C1
:10E02000F0C62000104078000080FB00E10F2000C7
:10E03000810F50002E003200F10F2000810F5000A0
:10E040004E003A0000C720001080FB0011C72000DE
:10E050009180FB00C808DD00010070000000E000B6
:10E0600043003A0040C720001080FB0051C7200049
:10E070009180FB00C808DD00010070000000E00096
:10E080003D003A000068EF0000C0EB0001E8B70077
:10E090000268EF000368EF0010C0B30012E8B70099
:10E0A000604180000000E000060032006041800016
:10E0B0009000780000002800008060000000E00070
:10E0C00007003A00E0C7200003C4B3000001780055
:10E0D0008040EB0010C0B3003BF9070040408800CF
:10E0E000E0C5200001C8B3000148780023003700D4
:10E0F00000C720001080FB0011C720009180FB00AA
:10E10000C808DD00010070000000E0001B003A00BC
:10E1100040C720001080FB0051C720009180FB0009
:10E12000C808DD0001007000E10F500013003A0044
:10E1300060C720008040EB000148780060C72000E5
:10E14000E06288001000200000638800E0C5200025
:10E1500011CCB30001487800000000000700370030
:10E160000000000005003700000000000300370039
:10E170000000000001003700000000000080FA00ED
:10E18000000006000200FA00114180000002200099
:10E19000808F5000020032000040EB00D7003700B3
:10E1A00000C8BF000080FB00E10F50008900320072
:10E1B000E10F500003003C000000E00006003200C8
:10E1C000BE003700E20F500088003200E30F50001D
:10E1D00098003200B9003700404080000000E000A5
:10E1E00006003200404080009000780000002800C7
:10E1F000008060000000E000B8003A000040EB0042
:10E20000004F780009003700C1EA20001E80FB00A3
:10E2100000804000E2C720009E80FB00810041009A
:10E2200091407800014878001E4FE8001E407800B9
:10E23000FE4F5000F4FF3600404080001040780050
:10E24000FF4F50005B003A006275800073758000DC
:10E250005035250021342400800F5100818F590052
:10E2600054003A0010C0B30012E8B70090EB200051
:10E27000104078000004E00046003A00A0EB2000C7
:10E2800010407800F04F500042003E00A0EB20000C
:10E29000104078000004E0003E00320080EB2000D7
:10E2A000104078008080FB00F003200000806000B8
:10E2B0000000E00037003A005035250021342500E9
:10E2C000F064880001658800807580009175800089
:10E2D00010658800216588006000B80030658800FE
:10E2E00041658800A0CA20008040EB00014878000A
:10E2F00000C0EB0001E8B7000268EF000368EF0020
:10E300000468EF00B0EB200010407800E34F5000AD
:10E310000A0032007176800000FF2F00008060004C
:10E320007076880080ED20008040EB000148780086
:10E3300090ED20008040EB000148780080EB200049
:10E34000104078000004E00003003D0010C0B3005E
:10E3500000E8B7000200370020C0B30000E8B700B3
:10E36000A0758000B1758000E00F5000E08F58006C
:10E37000020032001168EF000200370010C0B30045
:10E3800011E8B700B0EB20001040780001E8B700BA
:10E390000600370011C0B30010C0B300DDF807005D
:10E3A0008040EB0010C0B300DAF807000000000066
:10E3B0005100370011C0B30010C0B300D5F80700FA
:10E3C0008040EB0010C0B300D2F807001268EF00E5
:10E3D000490037004B000700E14F400041003A0080
:10E3E00030C0B30000E8B700430037004500070025
:10E3F000E14F40003D003A00A0CA200010407800E4
:10E400000004E00008003A003065800041658000AB
:10E41000E00F5000E08F580003003200A0CA200037
:10E4200021C0B3000148780030C0B30000E8B70055
:10E4300031003700804180000000E000060032001B
:10E44000804180009000780000002800008060007B
:10E450000000E00027003A00E0C92000D3C0B3006C
:10E460000001780011C0B30010C0B30056F80700D7
:10E4700050408800404080000000E000060032006C
:10E48000404080009000780000002800008060007C
:10E490000000E00007003A00E0C7200003C4B3001A
:10E4A000000178008040EB0010C0B30046F8070080
:10E4B000404088000068EF000F0037000068EF0060
:10E4C000A0CA200021C0B300014878008040EB00C2
:10E4D00010C0B3008FF807000700370000000000ED
:10E4E00005003700000000000300370000000000B6
:10E4F000010037000000000000C8BF000080FA00E3
:10E50000000006000000FA0021778000607780009C
:10E51000010001000004A2000004E00008003A002D
:10E5200090EB2000104078008080FB0000812000EC
:10E5300000804000104078000004E0000B00320032
:10E5400090EB2000104078000080FB0011002000BC
:10E550000008DD008080EA007040800000806000DC
:10E56000704088002D0007002900370090EB200044
:10E57000104078000080FB00110020008008DD00C2
:10E5800070408000008060000000E0001F003A0042
:10E59000F176800060778000010001000000E0005B
:10E5A0001800320090EB2000104078000080FB0043
:10E5B000110020008008DD00704080000100700024
:10E5C000704088007176800000FF2F00008060009E
:10E5D0006000B3007076880080ED200081C2B30037
:10E5E0000148780090ED20008040EB000148780061
:10E5F000A0CA200011C0B30001487800360007000F
:10E600000300370005000700010037003200070053
:10E6100001C8BF000080FA00000006000000FA00F8
:10E6200001C8BF000080FB00F20F50002100320043
:10E63000F20F500005003C000000E000170032001F
:10E64000E30F5000070032001E003700FE0F50009D
:10E6500012003200D10F2000810F5000170032004D
:10E66000180037001C0307007176800000FF2F00A0
:10E67000008060000010A0007076880080ED20000F
:10E68000A1C3B3000148780090ED20008040EB006A
:10E6900001487800100007000D003700A0CA2000D4
:10E6A00011C0B3000148780000C0EB0001E8B700DA
:10E6B00007003700080007000500370006000700C4
:10E6C00003003700F0C7B300C103070000000000DB
:10E6D0000080FA00000006000A00FA0001C8BF002E
:10E6E0000080FB00FE0F5000B2003200FE0F500011
:10E6F0000E003C00F20F50002C003200F20F5000D0
:10E7000005003C000000E000BE003200E30F5000B6
:10E710007200320024013700FA0F50008B003200E3
:10E72000FB0F5000CE0032001F013700A102200075
:10E73000810F500017003200A1022000810F50000D
:10E7400007003C0051022000810F500031003200D0
:10E7500081022000810F50000800320012013700B2
:10E76000F1022000810F5000BD003200D10F2000C7
:10E77000810F5000C00032000B0137003B01070041
:10E780000004E0000C013A0000C0EB0001E8B70013
:10E7900014013700E40107000004E00008013A001A
:10E7A00000C0EB0001E8B7000E01370011C8BF0040
:10E7B0000004E0000300320000C0EB0001E8B700F5
:10E7C00008013700E0EB20001040780015E8B700A2
:10E7D000F0EB20001040780014E8B700A040800063
:10E7E0008000EB00FC0207000004E000F6003A00A5
:10E7F00040022000FD0007004202200061D02900F5
:10E80000C0CA2000FBD30700D0CFB30001E8B70097
:10E81000F40037000177800060778000010001007C
:10E8200030079800410798001177800060778000DA
:10E83000010001008000EB001007980021079800FC
:10E840001E48900080407800C0CA2000014878002F
:10E850000E48900080407800D0CA2000014878001F
:10E860007E40900080407800E0CA20000148780097
:10E870006E40900080407800F0CA20000148780087
:10E880005E4090008040780000CB20000148780076
:10E890004E4090008040780010CB20000148780066
:10E8A0003E4090008040780020CB20000148780056
:10E8B0002E4090008040780030CB20000148780046
:10E8C00080002000A040880080002000C7000700D2
:10E8D000D0CFB30001E8B700C200370011C8BF00B5
:10E8E0000004E0000300320000C0EB0001E8B700C4
:10E8F000BC00370020012000A0408800200120003B
:10E90000BA0007000040EB00004F78000900370014
:10E910001E80FB001E81FB00C1EC20008100410035
:10E920009140780001417800C1CA200082707800CF
:10E930001E4FE8001E407800F14F5000F4FF3600F3
:10E94000D0CFB30001E8B700A6003700C0CA20004E
:10E9500031C0B30001487800D0CA20008040EB00ED
:10E960000148780041778000607780000100010055
:10E970000004E0000200320000C8B30001003700CC
:10E980000040EB00E1CA200080487800F0CA200077
:10E990008040EB000148780040002000A040880043
:10E9A0004000200091000700D0CFB30001E8B7007D
:10E9B0008C0037007176800000FF2F00008060001F
:10E9C0005000B3007076880080ED200001C2B300D3
:10E9D0000148780090ED20008040EB00014878006D
:10E9E000A0CA200011C0B300014878006000B80040
:10E9F000306588004165880000C0EB0001E8B70081
:10EA0000780037006000B800730207000004E000DF
:10EA10006F003A00E0EC2000104078006F4060008A
:10EA2000E64F500007003A00A0CA200010407800CE
:10EA3000E14F500003003A0000C0EB0001E8B700CE
:10EA400068003700240207006000B80030658800C5
:10EA50004165880000C0EB0001E8B70061003700A5
:10EA60006000B800306588004165880000C0EB0098
:10EA700001E8B7005B003700504080000000E00074
:10EA8000060032005040800090007800000028000E
:10EA9000008060000000E0004F003A00A275800096
:10EAA000B3758000F003200001002000800F5100AA
:10EAB000818F59000900360000C4B3001047980048
:10EAC000A0758000B17580000004B1000180B10024
:10EAD000A0758800B175880006003700A075800019
:10EAE000B1758000104798006000B800A0758800DC
:10EAF000B1758800A14080001E4090000080FB009E
:10EB0000808F500006003900A14080001E40900018
:10EB10000080FB0000805000A040880013003700F8
:10EB20000040EB00004F78000C003700A040800050
:10EB30000000E00004003200A04080000000E90076
:10EB4000A0408800040037001E80FB00C1CA2000DE
:10EB50000041EB00827078001E4FE8001E409000DC
:10EB60009E40780080CF5000F0FF3900C0CA2000DE
:10EB70009E4190000001780011C0B30010C0B300A6
:10EB800091F6070050408800A0758000B1758000A4
:10EB9000E00F5000E08F580011003A0000C0EB0079
:10EBA00001E8B7000F003700F0C7B3008802070084
:10EBB000000000000B0037000000000009003700D3
:10EBC00000000000070037000000000005003700CB
:10EBD00000000000030037000000000001003700C3
:10EBE000000000000080FA00000006000200FA00A9
:10EBF000000F7800A2758000B37580001E007800B9
:10EC00008000EB00800F5100818F59000800310017
:10EC10006000B8003065880041658800A0758000FC
:10EC2000B175800000007800A04088000D0037001A
:10EC3000A04080009E0F5000020036009E00780029
:10EC4000A1408800A2758000B3758000A0408000BC
:10EC50008000EB0000005100818059003065880081
:10EC6000416588000080FA00000006000000FA00FC
:10EC700002C8BF000080FB00E20F500033003200EA
:10EC8000E20F500005003C000000E00008003200E8
:10EC9000E10F50002300320093003700E30F5000D3
:10ECA00065003200E40F50006D0032008E00370026
:10ECB000D0EB20001040780019E8B700E0EB20000E
:10ECC0001040780018E8B700F0EB20001040780002
:10ECD00017E8B70000EC20001040780016E8B700F5
:10ECE00020EC20001040780015E8B70030EC200040
:10ECF0001040780014E8B700A04080006101B8001F
:10ED00004918DD00C710DE00810070004910DD00E9
:10ED1000B10107000004E0007B003A0010C0B3001E
:10ED200002E8B700A04080000000E00002003A00C6
:10ED30000268EF0079003700A04080000000E90081
:10ED4000A040880020C0B30002E8B7005040800017
:10ED50000000E00006003200504080009000780083
:10ED600000002800008060000000E00068003A0019
:10ED700034778000C1CA2000B2408000C3408000C8
:10ED80006077800004000100E14F50001C00320059
:10ED9000418020009140780030C6B30080CF500001
:10EDA00004003E0004C8BF000040E80004E8B700CB
:10EDB0005A003700A0CA200021C0B30001487800E3
:10EDC0007176800000FF2F00008060003000B300EB
:10EDD0007076880080ED20008040EB0001487800CC
:10EDE00090ED20008040EB000148780011C0B30096
:10EDF00010C0B30047F607000268EF004700370075
:10EE0000B0408000C140800061004000E0804800C8
:10EE1000B0408800C1408800002020000100200090
:10EE20003065880041658800C0CA200030408800F5
:10EE300030C0B30002E8B700306580004165800053
:10EE4000E00F5000E08F580003003A0010C0B300FC
:10EE500002E8B7003100370040C0B30002E8B70055
:10EE6000504080000000E00006003200504080006A
:10EE70009000780000002800008060000000E000A2
:10EE800025003A003040800003C4B3000001780040
:10EE900011C0B30010C0B300CBF50700504088008C
:10EEA00030C0B30002E8B700A0758000B1758000E3
:10EEB0000004B1000180B100A0758800B175880020
:10EEC00030658000416580000004B1000180B10020
:10EED0003065880041658800304080000004B00043
:10EEE000304088000D003700A0CA200021C0B300C8
:10EEF0000148780011C0B30010C0B30005F6070048
:10EF00000268EF0005003700000000000300370032
:10EF100000000000010037000000000002C8BF0030
:10EF20000080FA00000006000000FA0003C8BF00DD
:10EF30000080FB00E20F5000A0003200E20F500002
:10EF400005003C000000E00008003200E10F500026
:10EF50003C003200D0003700E30F50004600320082
:10EF6000E40F500072003200CB003700D0EB2000DD
:10EF70001040780019E8B700E0EB2000104078005E
:10EF800018E8B700F0EB20001040780017E8B70051
:10EF900000EC20001040780016E8B70020EC2000BC
:10EFA0001040780015E8B70030EC200010407800E1
:10EFB00014E8B700A04080006101B8004918DD00E6
:10EFC000C710DE00810070004910DD00020107005B
:10EFD0000004E000B8003A004177800060778000CC
:10EFE000010001000004E00014003200A0CA20006B
:10EFF00011C0B300014878007176800000FF2F0037
:10F00000008060007000B3007076880080ED200002
:10F0100071C2B3000148780090ED20008040EB0001
:10F02000014878008040EB0010C0B300B9F507003C
:10F030000368EF0003C8BF00A500370010C0B3008D
:10F0400000E8B700A04080000000E00002003A00A5
:10F050000368EF009D00370030C0B30003E8B7003D
:10F06000C0CA20003040880000202000010020009D
:10F07000306588004165880030658000416580000A
:10F08000E00F5000E08F5800130032004040800035
:10F090000000E00006003200404080009000780050
:10F0A00000002800008060000000E00084003A00BA
:10F0B0003040800003C4B300000178008040EB00C2
:10F0C00010C0B30040F507004040880040C0B300C6
:10F0D00003E8B700160037004177800060778000B2
:10F0E000010001000004E0000E003200A0CA200070
:10F0F00011C0B300014878007176800000FF2F0036
:10F10000008060000010A0007076880080ED200074
:10F1100071C2B3000148780090ED20008040EB0000
:10F120000148780020C0B30003E8B700670037004B
:10F13000404080000000E0000600320040408000B7
:10F140009000780000002800008060000000E000CF
:10F150005D003A00A2758000B375800040408000D9
:10F16000104078000080FB008000EB0000005100A0
:10F1700081805900A0758800B175880032658000D3
:10F180004365800040408000104078000080FB0014
:10F190008000EB000000510081805900306588003C
:10F1A00041658800304080000004B0003040880095
:10F1B00030C0B30003E8B70044003700A0CA200005
:10F1C000104078000004E00027003A0055778000E6
:10F1D000B0408000C14080000080700000F0A700B7
:10F1E0000000EA000000E9004F00DE000042780065
:10F1F000C1CA2000B2408000C34080006077800018
:10F2000005000100E14F500017003200418020004E
:10F210009140780030C6B30080CF500004003E001B
:10F2200004C8BF000040E80004E8B700270037002A
:10F23000A0CA200011C0B300014878007176800098
:10F2400000FF2F00008060003000B300707688005F
:10F2500080ED20008040EB000148780090ED200018
:10F260008040EB0001487800B0408000C140800041
:10F2700061004000E0804800B0408800C140880044
:10F28000A04080000000E900A040880010C0B3004A
:10F2900003E8B7000D003700A0CA200021C0B3006A
:10F2A000014878008040EB0010C0B30019F507005A
:10F2B0000368EF000500370000000000030037007E
:10F2C00000000000010037000000000003C8BF007C
:10F2D0000080FA00000006000000FA00617680005D
:10F2E00000F82F00808060000007200001007000FF
:10F2F00060768800607680000070A10060768800EB
:10F30000D0EC20008040EB0001487800717680004E
:10F3100000FF2F000080600070768800707680000B
:10F320000050A10070768800707680000060A10017
:10F3300070768800707680000070A100707688007A
:10F34000F0EC20008040EB000148780000ED200048
:10F350008040EB000148780010ED20008040EB0079
:10F360000148780020ED20008040EB000148780043
:10F3700030ED2000A1C0B300014878006000B80063
:10F38000A0768800B176880080ED20008040EB00F8
:10F390000148780090ED20008040EB0001487800A3
:10F3A000A0ED20008040EB0001487800B0ED200087
:10F3B0008040EB0001487800C0ED20008040EB0069
:10F3C00001487800D0ED20008040EB000148780033
:10F3D0000080FA00000006000800FA0020079800EC
:10F3E000310798002E009000BE009000E00F500002
:10F3F000E08F580003003A0010C0B3002047980087
:10F40000020037000040EB002047980011C8BF0001
:10F410000004E000050032002E4090000004E000EF
:10F42000020032000040EB0067003700A275800048
:10F43000B37580002E009000BE009000800F510038
:10F44000818F590011003A0000C8BF00E14F500001
:10F4500007003A001180200091407800A0C2B3005C
:10F4600080CF5000090032000040EB00560037000A
:10F470001180200091407800A0C2B30080CF5000DE
:10F4800002003A000040EB004F003700A2758000F8
:10F49000B37580002E009000BE009000800F5100D8
:10F4A000818F59000300360010C0B3001047980048
:10F4B000020037000040EB001047980000C8BF0072
:10F4C000E24F500021003A00118020009140780066
:10F4D000A0C2B30080CF5000070032002E40900041
:10F4E0000004A2000004E0000300320050C0B3009A
:10F4F000004F78003100370011C8BF000004E00061
:10F500000300320010C0B300004F78002B0037001A
:10F510002E4090000004E0000300320040C0B30021
:10F52000004F7800250037001E4090000004E000E6
:10F530000300320040C0B300004F78001F003700C6
:10F5400050C0B300004F78001C003700118020002D
:10F5500091407800A0C2B30080CF500003003A0071
:10F5600030C0B300004F78001400370011C8BF004E
:10F570000004E0000300320010C0B300004F780028
:10F580000E0037002E4090000004E000030032001F
:10F5900020C0B300004F7800080037001E409000E4
:10F5A0000004E0000300320020C0B300004F7800E8
:10F5B0000200370030C0B300004F78001E407800D2
:10F5C000030007001E4078000080FA0000000600DB
:10F5D0000400FA0020479800504080000000E0003E
:10F5E00006003200504080009000780000002800A3
:10F5F000008060000000E00063003A0040408000AE
:10F600000000E000060032004040800090007800DA
:10F6100000002800008060000000E0005C003A006C
:10F620000180200091407800014F780000C0EB007D
:10F6300001E8B7000268EF000368EF00A0758000E2
:10F64000B17580003065880041658800A0CA20003F
:10F6500011C0B3000148780030C0B30000E8B70023
:10F660002E4090000080FB00E30F50001700320096
:10F67000E30F500005003C00E10F50000B0032008A
:10F68000E20F50000D00320042003700E50F50003D
:10F6900019003200E50F500013003500F10720007B
:10F6A000810F50001B0032003A003700A0CA200032
:10F6B00021C0B300014878003600370011C0B30004
:10F6C00010C0B30013F4070032003700A0CA2000B6
:10F6D00021C0B3000148780011C0B30010C0B300CE
:10F6E0000CF407002B0037008040EB0010C0B30083
:10F6F00008F4070027003700A0CA200021C0B3008B
:10F70000014878008040EB0010C0B30001F407000E
:10F7100020003700F0FE07007176800000FF2F0008
:10F72000008060005000B3007076880080ED2000FB
:10F7300001C2B3000148780090ED20008040EB004A
:10F74000014878001E407800E24F50000A003A005D
:10F75000A0758000B1758000E00F5000E08F580068
:10F76000050032008040EB0010C0B300E9F3070051
:10F77000000000000700370011C0B30010C0B30044
:10F78000E4F3070003003700000000000100370029
:10F79000000000000080FA00000006000200FA00ED
:10F7A000000F780012C8BF000004A2000004E000AF
:10F7B0000700320011C0B30010C0B300D5F307003A
:10F7C0008040EB0010C0B300D2F307000A003700FE
:10F7D000604180009E0F500007003A00E0C7200003
:10F7E00003C4B300000178008040EB0010C0B300F8
:10F7F00075F30700404088000080FA000000060012
:10F800000000FA00A20007000040FE005124800022
:10F8100000022000008060000000E00002003A00CA
:10F8200010C0B30041000700D200070010C0B300B1
:10F830000080FA00000006000000FA0036C8BF0091
:10F840000004E0003600320037C8BF000004E000CA
:10F850003300320040248000620060000000E000BD
:10F86000010032008824A900750007000004200070
:10F870000024880000000000012480000004200013
:10F88000008060000000E000FBFF32000004200068
:10F8900000248800000000000124800000042000F3
:10F8A000008060000000E000FBFF32000004200048
:10F8B00000248800000000000124800000042000D3
:10F8C000008060000000E000FBFF32009444A800CC
:10F8D00000042000002488000000000001248000B3
:10F8E00000042000008060000000E000FBFF320008
:10F8F0000004200000248800000000000124800093
:10F9000000042000008060000000E000FBFF3200E7
:10F910009444A9005700070010C0B300010037004D
:10F920000040EB000080FA00000006000400FA002E
:10F930002047980040248000610060000000E00043
:10F940000B00320040248000620060000000E000F4
:10F9500007003A0046C8BF00E34F500004003600DD
:10F96000202480004300DE00614060003200370048
:10F970002E4090000004E0001D0032008824A90001
:10F980008804A8002E0007000040EB00004F78001C
:10F990000900370000042000002488000000000057
:10F9A0000124800000042000008060000000E000CE
:10F9B000FBFF32001E4FE8001E407800E44F50006D
:10F9C000F4FF36000040EB00104798002024800030
:10F9D000680060000000E0000200320010C0B300C8
:10F9E00010479800230007001E40900012003700C7
:10F9F00040248000610060000000E00002003A0046
:10FA000000C0EB000C003700402480006200600062
:10FA10000000E00002003A00E0CFB300060037002B
:10FA200046C8BF00E34F500002003E00D0CFB300F5
:10FA300001003700C0CFB3000080FA0000000600CC
:10FA40000000FA005068EF001000FC00F104800094
:10FA500000042000008060000000E000020032008E
:10FA600010C0B30050E8B7009EC0A9000080FA00A3
:10FA7000000006000000FA0050C8BF000004E000CB
:10FA8000010032009EC0A8000080FA0000000600BD
:10FA90000400FA001E00FC0011028000000E20008D
:10FAA000008060004042880011028000000E2000AB
:10FAB0000100700010028800400920001007980023
:10FAC0000000EB00000F78000E0037001E009000D1
:10FAD000900078001E0078000001400020EF200018
:10FAE00000004100010878001E0090008000EB003B
:10FAF000010878001E0090000080E80010079800C0
:10FB00001E0FE8001E007800E50F5000EFFF3600E2
:10FB100060248000504288008C24EF001024800074
:10FB2000604288008224EF00700680004800DE00FA
:10FB3000674060000080FB007042880000012000E8
:10FB40000024880000022000502488008EC0A900F4
:10FB50008284A80071068000F08F2F000080600072
:10FB600000A0A000700688009EC0A8000080FA00D7
:10FB7000000006000400FA00400920001007980069
:10FB80000000EB00000F78000B0037001E0078002B
:10FB90008000400020EF20000080400090007800AE
:10FBA0001E009000010878001E0090000080E80010
:10FBB000100798001E0FE8001E007800E50F5000A7
:10FBC000F2FF3600504280006024880060428000CE
:10FBD0001024880070428000004078006740600078
:10FBE0000080FB00670060004800DD0072068000B6
:10FBF000F18F2F0081006100010070007006880005
:10FC000011028000F0F12F008080600040428000EF
:10FC100001007000404288004042800010028800CD
:10FC20000080FA00000006000000FA0001178000C2
:10FC300000F02F000080600000178800F002A9008B
:10FC4000F022A900E822A900F402A900F422A900E8
:10FC5000EC22A90000502300C1002000620107002F
:10FC60008040EB0080C3B300110007008040EB0030
:10FC700080C0B3000E0007008040EB0010C0B3004E
:10FC80000B0007008040EB0060C0B30008000700D5
:10FC90008040EB00C0C0B3000500070000B82B0097
:10FCA00001002000500107000080FA00000006005B
:10FCB0000400FA002047980031479800011780009F
:10FCC000F00F20000100700000178800F422A80047
:10FCD000F402A9002117800000F02F0000806000CE
:10FCE00020178800EC22A80000000000000000009F
:10FCF00000000000101780004700DE006140600037
:10FD0000004F7800EC22A9001E4078000004E000BB
:10FD1000F4FF3A000117800000F02F00008060001F
:10FD200000178800F422A9003E4090000080FB00EC
:10FD30000000EA004F00DE00004078000080FB0079
:10FD400061006000A11780000100A10001007000A7
:10FD5000A01788002117800000F02F00808060002D
:10FD60002E4090000080FB000100700020178800EA
:10FD7000EC22A800000000000000000000000000CD
:10FD8000EC22A9000080FA00000006000400FA003E
:10FD9000100798008F0037001E009000104F780069
:10FDA0001E00FB006101B9000005200001002000D9
:10FDB0000200400083804800C204200003002000AD
:10FDC000820F5000838F580075003E0000600100D4
:10FDD0007000370072003700710037007000370084
:10FDE0006F003700680037006D0037006C00370087
:10FDF0006B0037006A003700690037006800370081
:10FE00006700370066003700650037006400370080
:10FE10006300370062003700610037006000370080
:10FE20005F0037005E0037005D0037005C00370080
:10FE30005B0037005A003700590037005800370080
:10FE40005700370056003700550037005400370080
:10FE50005300370052003700510037005000370080
:10FE60004F0037004E0037004D0037004C00370080
:10FE70004B0037004A003700490037004800370080
:10FE8000470037004600370045003700380037008C
:10FE9000430037001B0037004100370040003700A7
:10FEA0003F0037003E0037003D0037003C00370080
:10FEB0003B003700160037003900370038003700A4
:10FEC00037003700150037003500370034003700A1
:10FED0002A003700320037003100370012003700A7
:10FEE0002F0037001C0037001E0037002C003700A1
:10FEF0002B0037002A0037000E00370013003700B0
:10FF00000F0037000040EB00004F7800240037005E
:10FF100010C0B300004F78002100370020C0B300AC
:10FF2000004F78001E00370030C0B300004F78004B
:10FF30001B00370040C0B300004F780018003700A6
:10FF400050C0B300004F78001500370060C0B30008
:10FF5000004F78001200370070C0B300004F7800E7
:10FF60000F003700F0CEB300004F78000C003700D0
:10FF700080C0B300004F78000900370090C0B30084
:10FF8000004F78000600370040CEB300004F7800E5
:10FF900003003700F0CDB300004F780000000000F0
:10FFA0001E407800EA4F500004003A008040EB0009
:10FFB00000CCB3003EFF0700030037001E4078006E
:10FFC00011C0B3003AFF07001E0090000000E800D7
:10FFD000100798001E009000104078000004E00018
:10FFE0006DFF3A000080FA00000006000200FA00EF
:10FFF0008040EB0000C4B3002DFF07000000EB00C1
:020000040001F9
:10000000000F780006003700E0CA29001E004000FB
:100010001040780011C0B30025FF07001E0FE80054
:10002000F00420009E007800808F5000F6FF34001E
:100030008040EB0000C8B3001DFF07000080FA00FD
:10004000000006000600FA00000F78001107980073
:10005000220798001E00780021072000810F500021
:100060001D00320021072000810F50000C003C00D1
:10007000E20F50001A003200E20F500003003C0073
:10008000E10F50000D0032001A003700E30F50005E
:100090000C003200E50F50000C0032001500370054
:1000A00041072000810F50000F003200410720005F
:1000B000810F50000E0035000E003700ADCF070055
:1000C0000C003700CCF707000A0037001E00900034
:1000D000B2FD0700070037000000000005003700F0
:1000E000000000000300370000000000010037009E
:1000F0000000000010C0B3000080FA0000000600FD
:100100005C0C00005002000000000000220800000B
:100110002600000000000000001000002000000089
:1001200000000000F20E00000C00000000000000C3
:10013000480800000A00000000000000AC0E0000AB
:100140003200000000000000000800002200000053
:1001500000000000DE0E000014000000020000009D
:10016000641D4E001D441D003A1D82001DB01F007D
:10017000001E000000000000000000005208000007
:100180000A000000000000005C08000000040000FD
:1001900000000000000000000000FA008BCF070004
:1001A00097EF0700A0FE070090FF0700A0D22900EC
:1001B000F6FE07000CF0070010418000FF0F500012
:1001C00001003E000700370040248000620060000C
:1001D0000000E00001003200020037006CCF070091
:1001E000F4FF3700F3FF3700F03FB1000180B100AA
:1001F00006003500EE03090000000000403FB1009A
:100200000180B100FBFF3D001000B000203FB000B6
:100210000200350000800900000000000000060018
:020000040002F8
:020000040003F7
:020000040004F6
:020000040005F5
:1057F000FFFF0000FFFF0000B62300007F3E000017
:00000001FF
